:020000040800F2
:100000003034002019010008CB010008C3010008AA
:10001000C7010008A10100087D02000800000000DF
:10002000000000000000000000000000F7010008D0
:10003000C101000800000000F5010008F9010008F6
:1000400033010008330100083301000833010008C0
:1000500033010008330100083301000833010008B0
:1000600033010008330100083301000833010008A0
:100070003301000833010008330100083301000890
:100080003301000833010008330100083301000880
:1000900033010008A50100083301000833010008FE
:1000A0003301000833010008330100083301000860
:1000B0003301000833010008330100083301000850
:1000C0003301000833010008330100083301000840
:1000D0003301000833010008330100083301000830
:1000E000330100083301000833010008000000005C
:1000F0000000000000000000000000000000000000
:1001000033010008DFF80CD000F038F80048004751
:100110009908000830340020064880470648004708
:10012000FEE7FEE7FEE7FEE7FEE7FEE7FEE7FEE7A7
:10013000FEE7FEE7190200080501000840EA010396
:100140009B0703D009E008C9121F08C0042AFAD28D
:1001500003E011F8013B00F8013B521EF9D2704751
:1001600010B5002200E0521C835C8C5CA34201D1DC
:10017000002BF8D1D8B2E1B2401A10BD064C074DA1
:1001800006E0E06840F0010394E807009847103467
:10019000AC42F6D3FFF7BAFF14190008341900086F
:1001A00000BFFEE710B5012000F08CFF0348006897
:1001B00040F020000149086010BD000010640040BC
:1001C000704700BFFEE700BFFEE7704710B500288C
:1001D00007DA0A07140E054A00F00F031B1FD45458
:1001E00003E00A07130E024A135410BD18ED00E095
:1001F00000E400E07047704705480068401C04496F
:10020000086004480068401C02490860704700000C
:10021000000000200400002010B51448006840F0E1
:1002200001001249086008464068114908400F491A
:100230004860084600680F4908400C4908600846B5
:10024000006820F480200860084640680A49084099
:1002500006494860084600680649084003490860A6
:100260004FF41F00886000F0C7FC10BD0010024072
:100270000C00FFE8FFFFF6FEFFFF00F700BFFEE700
:1002800002E008C8121F08C1002AFAD1704770475F
:10029000002001E001C1121F002AFBD1704770B598
:1002A00006460C46154605EB8500810004F1080062
:1002B000405820F0010105EB8500820004F10800A0
:1002C0008150182105EB8500820004F10C0081505B
:1002D00005EB8500810004F10800405840F0010161
:1002E00005EB8500820004F108008150304601F0E2
:1002F000D3FA70BD10B500BF032206490648FFF7C8
:10030000CEFF00BF00BF062202490448FFF7C7FF27
:1003100000BF10BD00000240003801400044004012
:1003200070B588B006460C46154601208DF81E00B3
:100330002548039001208DF81D000020049018200E
:100340000590301D019000208DF81C0002904FF4A4
:100350004050069001AA2946204600F03FF905EBDF
:100360008500810004F10800405820F0200105EBD1
:100370008500820004F1080081504FF41641304698
:1003800001F03AFA0021304601F0BBFA0021304674
:1003900001F0A7FA0021304601F093FA002130461F
:1003A00001F087FA0021304601F07BFA0421304643
:1003B00001F08FFA0821304601F09BFA8021304687
:1003C00001F062FA08B070BD4200002010B500BF15
:1003D00040F20E6000F0F0FA40F2026000F0ECFA39
:1003E00040F2026000F0E8FA4FF4A06000F0E4FA96
:1003F00040F20E3000F008FC40F20E3000F0ECFA53
:100400004FF40073032218211D4800F08DF94FF4BA
:100410008063032204211A4800F086F90322194957
:100420001948FFF77DFF00BF00BF40F2117000F0D8
:10043000C3FA40F2026000F0BFFA40F2026000F03E
:10044000BBFA4FF4A06000F0B7FA40F2114000F0A0
:10045000DBFB40F2114000F0BFFA04230322182115
:10046000074800F061F9082303220421044800F042
:100470005BF9062203490548FFF752FF00BF10BD94
:1004800000080140000002400038014000440040E4
:1004900030B5034688189C8890FBF4F504FB1500E2
:1004A00080B230BD38B5044601226946204600F0CE
:1004B00031F8002802DD9DF8000038BDFF20FCE780
:1004C00070B504460E4615462660A580204600F00D
:1004D00001F870BD10B503680279002102E059549B
:1004E0004C1CE1B29142FADB541E04810024C4800A
:1004F00010BD13B50446012201A9204600F032F8D0
:100500001CBD70B504460D46E1882A462046FFF71B
:10051000BFFF70BD2DE9F04105460C461646274643
:1005200004EB060811E0E8882989884203D1E01B22
:1005300080B2BDE8F081E9882868405C2070012124
:100540002846FFF7DEFFE880641C4445EBD33046C5
:10055000EFE770B504460D4621892A462046FFF78D
:1005600097FF70BD2DE9F04705460C461646274615
:1005700004EB060912E001212846FFF7EAFF804656
:10058000E888404503D1E01B80B2BDE8F0872078C1
:100590002A8929688854A5F80880641C4C45EAD348
:1005A0003046F2E713B50446012201A92046FFF7C1
:1005B000D9FF1CBD10B504460548844207D140F25E
:1005C000194000F021FB40F2194000F005FA10BD7F
:1005D0000064004042690A43426170472DE9F041DE
:1005E00004460D4616462946204600F08FF808B905
:1005F00000BFFEE705EB8500820004F110003168C2
:10060000815005EB8500820004F11400B16881502F
:10061000308A81B205EB8500820004F10C00815024
:1006200005EB8500810004F10800475827F47C574A
:10063000F1687068084371690843074305EB85005A
:10064000810004F108004750307E01280ED105EBEF
:100650008500810004F10800405840F0400105EB9E
:100660008500820004F1080081500DE005EB850053
:10067000810004F10800405820F0400105EB85009E
:10068000820004F108008150707E01280ED105EB34
:100690008500810004F10800405840F0800105EB1E
:1006A0008500820004F1080081500DE005EB850013
:1006B000810004F10800405820F0800105EB85001E
:1006C000820004F108008150B07E70B905EB85000E
:1006D000810004F10800405820F0100105EB85006E
:1006E000820004F1080081500DE005EB85008100D7
:1006F00004F10800405840F0100105EB850082002D
:1007000004F108008150BDE8F0810000024601209C
:10071000034B9A4202D1042900DD002070470000FB
:100720000004024041617047F0B5044616460025BA
:10073000002201F00F0501F0100707B1354300203A
:100740001EE0012787401F40C7B122684FEA800C96
:100750000F2707FA0CF7BA43870005FA07F73A4361
:10076000282904D1012787401F40676105E04829F7
:1007700003D1012787401F4027612260471CB8B280
:100780000828DED3082022E0012787401F40E7B178
:100790006268A0F108074FEA870C0F2707FA0CF7E9
:1007A000BA43A0F10807BF0005FA07F73A43282922
:1007B00004D1012787401F40676105E0482903D124
:1007C000012787401F4027616260471CB8B210288C
:1007D000DAD3F0BD00F01F0201219140024A43111B
:1007E00042F823107047000080E100E00249014315
:1007F000024A1160704700000000FA050CED00E0AD
:100800005053313030000000F0B50A460023002478
:100810000021002500F00046B6F1004F02D11D4E28
:10082000F16901E01B4E7168C0F3034583B200F427
:100830004016B6F5401F08D121F07061154E76685C
:1008400026F07066134F7E6012E000F48016B6F555
:10085000801F06D1032606FA05F4A14341F070611A
:1008600006E0460D360103FA06F6B14341F0706129
:1008700022B1460D360103FA06F6314300F0004678
:10088000B6F1004F02D1034EF16101E0014E7160FB
:10089000F0BD00000000014008B53CA000680090D9
:1008A0000025012000F0A8FD40F2026000F084F86D
:1008B00040F2036000F080F840F2046000F07CF841
:1008C00040F2056000F078F840F2066000F074F83D
:1008D00000BF2F4800680A21B0FBF1F4601EB0F1A0
:1008E000807F00D30FE0601E4FF0E02148610F21B0
:1008F0004FF0FF30FFF76AFC00204FF0E0218861E5
:100900000720086100BF0021481EFFF75FFC00BF01
:10091000FFF75CFD00F088F9032269467F2000F0B4
:100920003BFC32E000F08AFA1A4800681E2804D91D
:10093000002018490860FFF7DDFC17480068B0F593
:10094000167F22D9002014490860681CC0B20546F1
:100950000A2810DD00BFBFF34F8F1048006800F475
:10096000E0600F490843001D0C490860BFF34F8F3A
:1009700000BF00BFFEE7002000F03EFD00F054F98C
:10098000032269467F2000F007FCCBE7F04200001D
:100990005C00002000000020040000200CED00E0BE
:1009A0000000FA05024A0A400243024B1A607047EF
:1009B00080FFFF1F08ED00E0064A02EB9011096876
:1009C00000F01F0301229A401143024B03EB9012E7
:1009D0001160704700100240064A02EB901109684E
:1009E00000F01F0301229A409143024B03EB901247
:1009F000116070470010024001700A124270704787
:100A00004C6F616465725F5632303230303531344C
:100A1000000000002DE9F04103460D461646002473
:100A20000027A0462448006800F4E060B0F5A06FFD
:100A300015D006DCB0F5407F18D0B0F5806F19D125
:100A400010E0B0F5C06F06D0B0F5E06F12D100270E
:100A50004FF0040815E001274FF0030811E00227CA
:100A6000B8460EE003274FF001080AE004274FF0D4
:100A7000000806E04FF4A060FFF7B8FE0227B84672
:100A800000BF00BFC7F1040005FA00F4C8F104017B
:100A90000F20C8403040044324010848C45403F0E8
:100AA0001F01012088405911890001F1E021C1F89E
:100AB0000001BDE8F08100000CED00E000E400E082
:100AC0002DE9F04F8BB00746002009903EA090E83A
:100AD000004CC068CDE905BECDF810A007900FF21C
:100AE000EC0ADAE9000ACDE9020A0FF2E00ADAE9D3
:100AF000000ACDE9000A38484068C0F381000A9036
:100B00000A9820B1012804D0022829D103E03349F2
:100B100028E0324926E03048406800F48038B8F5D3
:100B2000803F09D12D4C2C48406800F40039B9F5BC
:100B3000003F02D1641000E0294C27484068C0F310
:100B400083422548406800F0006008B142F010027E
:100B50000F2A01D2921C00E0521C04FB02F101E0BA
:100B60001E4900BF00BF1C484068C0F3031504A81D
:100B7000465D21FA06F318484068C0F3022502A832
:100B8000465D23FA06FC14484068C0F3C2251DF8F0
:100B9000056023FA06F0089037B1012F06D0022F26
:100BA00006D0032F0AD106E0099108E0099306E078
:100BB000CDF824C003E00898099000E000BF00BF12
:100BC00009980BB0BDE8F08F0000000000000000A5
:100BD00001020304060708090010024000127A000F
:100BE00000093D0010B51520FFF7F4FD0148FFF79F
:100BF000E1FC10BD0064004010B500F0A7FD10BD81
:100C0000426F6F7400000000064A02EB9011096801
:100C100000F01F0301229A401143024B03EB901294
:100C2000116070470010024010B500BF0622244931
:100C30002448FFF745FC0B2223492448FFF740FCDA
:100C400040F20360FFF7B8FE4FF4C060FFF7B4FE58
:100C500040F21970FFF7B0FE00BF00BF4FF4807381
:100C6000032248211A48FFF75FFD4FF40073032267
:100C700018211748FFF758FD01214FF4EA10FFF73C
:100C8000C3FD40F20260FFF797FE4FF48051114818
:100C9000FFF748FD4FF48053032210210D48FFF762
:100CA00043FD80210B48FFF73DFD802303221021E7
:100CB0000848FFF739FD00BF00F072F810BD0000D2
:100CC0000D000020001000200C1000201810002043
:100CD000000C01400008014030B50B46012404FA25
:100CE00000F1234C246844F00104214D2C60204C79
:100CF0001C3424688C431E4D1C352C601C4C0C3459
:100D000024680C431A4D0C352C60042404EBC204F7
:100D1000A4B2174D403545F830404FF47F7405EBD1
:100D2000C0056C60124C241D24688C43104D2D1D91
:100D30002C603BB90E4C143424688C430C4D143594
:100D40002C6006E00A4C143424680C43084D14351A
:100D50002C60074C1C3424680C43054D1C352C605A
:100D6000034C246824F00104014D2C6030BD0000C8
:100D7000006600400948016801F0806008B1002069
:100D8000704701F0006008B10120F9E701F08050E0
:100D900008B10220F4E70320F2E7000008640040F5
:100DA00010B52448FFF706FC2248006820F0020036
:100DB000204908600846006840F0010008604FF6CE
:100DC000FF7400E0641E1B48001D006800F0010075
:100DD00008B9002CF6D1184816491C31086015488E
:100DE000006820F0E800134908600846006840F0F9
:100DF000140008600846006820F0010008604FF603
:100E0000FF7400E0641E0B48001D006800F0010044
:100E100008B1002CF6D1422201210020FFF75CFF2F
:100E2000002211461520FFF7F5FD10210148FFF7BC
:100E3000D1FB10BD006400401700240038B51248F3
:100E4000006800F0040008B1FFF7AAFF00F01EFAE6
:100E500012E09DF8000000EB40100C4901EBC004CB
:100E6000E288607804F1080100F016F800BF9DF8F0
:100E700000100748FFF73DFB012269460548FFF7D0
:100E800049FB0028E5DC38BD1864004088050020D7
:100E900018100020280000202DE9F74F82B0894665
:100EA0001746B9F8000001904FF6F071019808401C
:100EB00044F2F021884202D005B0BDE8F08F002056
:100EC0004A49086009F10205B81E87B20198A0F5E9
:100ED0008440F038092875D2DFE800F005071024B7
:100EE00029485174550000246FE000BF002040499C
:100EF000086000F0BBFB002400BF66E02E463046D1
:100F000000F05AFA8046F01C00F05FFA8246514623
:100F1000404600F0B9FB08B1002001E04FF0FF307F
:100F2000044652E03946284600F06CFBC4E72E46E2
:100F3000B846304600F040FA82462D4800685045D9
:100F40000CD1A8F103001FFA80F84146F01C00F014
:100F500059FB274800684044254908602448016837
:100F6000701C00F03EFA032400BF2EE0002000F0C9
:100F700043FA08B1002401E04FF0FF3425E00120DE
:100F80006870012421E0A8463E46404600F014FA6D
:100F900083460BF1006A002601E0701C86B21AF845
:100FA000060008B1FA2EF8DB594608F1010000F0FE
:100FB00018FA3246514608F10400FFF7BFF8F41C56
:100FC00003E0FFE74FF0FF3400BF00BF002C03DA5F
:100FD00000240120287001E000202870E01C82B26B
:100FE0004946029800F046F900BF65E7040000207A
:100FF000340000202DE9F0410546884600260AE02D
:10100000184850F826406078A84202D12046BDE832
:10101000F081701CC6B2144800788642F0DB12489A
:1010200000780A2817D21148FFF73CFA0746FF2F2D
:1010300001D10020EBE707EB47100D4901EBC0049D
:1010400008480949097840F8214007480078401CC1
:101050000549087001E0034804686570FF20E070EE
:101060002046D4E7D80F00200C00002018100020E4
:1010700088050020024600211AE0104850F821009F
:10108000904213D10E480078401E0D4B187007E0B7
:101090000A4B481C53F8200043F82100481CC1B2F9
:1010A000074800788142F3DB01207047481CC1B239
:1010B000034800788142E0DB0020F6E7D80F0020EB
:1010C0000C0000202DE9F05F0646304901EB0610C8
:1010D000D0F8B0A50AF00600042802D00120BDE82F
:1010E000F09F4FEADA05294901EB0610D0F8B4A5C4
:1010F000C5F38437C5F3C4484146C5F3C610FFF7AE
:1011000079FF04460CB90020E9E7E078B8420ED038
:10111000012F01D00120E2E7C5F30160A07005F0C6
:101120007F0020700020E0800220E07003E0781C47
:1011300000F01F00E070E18804F1080001EB0009F5
:10114000E0880AF00F010844E080104901EB061026
:10115000D0F8B805C9F8000001EB0610D0F8BC05BE
:10116000C9F80400B8450ED10948201A4FF484711B
:1011700090FBF1F000F0FF0B59460648FFF712FA1A
:101180002046FFF777FF0120A9E70000006000403C
:101190008805002028000020F8B506460C461546B4
:1011A0002346012242213046009500F031F8F8BD77
:1011B00070B5164D05EB0014D4F8844524F00F04E7
:1011C0002E4606EB0015C5F88445354605EB0014A0
:1011D000D4F884451C4306EB0015C5F8844506EB9E
:1011E00000151468C5F88845042B04DD06EB0015CE
:1011F0005468C5F88C456FF0070404EAC104641D07
:10120000024E06EB0015C5F8804570BD0060004039
:101210002DE9F04706460F4690469946DDF820A096
:101220001148FFF73FF90546FF2D02D10020BDE828
:10123000F08705EB45100D4901EBC0040020A080AC
:1012400084F8028026706770A4F806A052464946CA
:1012500004F10800FEF772FF29460548FFF7A2F9DE
:1012600000F014F80120E2E70010002060000020E8
:101270001C000020F8B506460C46154623460222FF
:10128000422130460095FFF7C3FFF8BD38B532E084
:101290001A480068C8B11948006880881749096869
:1012A000C988884204DA1548006800F02FF823E066
:1012B000124800681249401A4FF4847190FBF1F013
:1012C000C4B221460F48FFF714F9012269460E48BF
:1012D000FFF720F9002809DD9DF8000000EB401021
:1012E000074901EBC0000549086003E000200349FD
:1012F000086001E000BFCBE700BF38BD0800002058
:1013000060000020001000201C0000202DE9F047A4
:101310000446FFF72FFD8046B8F1030F12D1244891
:1013200000682449884205D9FFF73AFD002020498A
:10133000086004E01E480068401C1D490860002049
:10134000BDE8F087E188C81DC11700EB5171C1F3FA
:10135000C706A088C11700EB5171C910491CCFB254
:10136000A0784FF0C05141EA006006F01F0140EA4A
:10137000C14007F01F0140EA8130217808436178BD
:1013800040EAC119E088A188401A85B2082D00DD25
:101390000825EBB2A18804F108000A184946404626
:1013A000FFF706FFA0882844A0800120C8E70000BE
:1013B0003800002040420F00014608784A7840EA91
:1013C00002208A7840EA02407047014608784A784D
:1013D00040EA02208A7840EA0240CA7840EA026085
:1013E000704710B504460B4699B22046FFF704FB40
:1013F000180CA07010BD0000FEB5064600F0B4F851
:101400000446314D314F32A13846FEF7A9FE08B1EE
:101410000020FEBDA868401CF8B92F4802902E4954
:10142000A068884211D02868401C20B1286800902C
:101430006868019003E020680090606801900123D3
:101440000C226946204600F045F90023042202A937
:1014500005F1080000F03EF900BF2EB11E49A0685A
:10146000884219D00020D4E700F038F8A0F50050E9
:101470002168884206D22068401C08B90120C8E7CC
:101480000020C6E710481030216800F02FF861688E
:10149000884201D00020BCE7FFF7A4FB00204FF0FA
:1014A000E021086108491031086880F3088800BF0E
:1014B000002105481030FFF775FA034910314868DC
:1014C00080470020A5E70000F01F00080028000862
:1014D000505331303000000044332211024800687C
:1014E0000004800970470000E0F7FF1FF0B50346D5
:1014F0000C464FF0FF311A46161912E010780025FD
:101500000CE081EA000707F001071FB1074F87EAE7
:10151000510100E0490840106F1CFDB2082DF0DBBE
:10152000521CB242EAD3C843F0BD00002083B8ED9C
:1015300010B50446A2B2012308490948006800F02A
:10154000C9F808B9002010BD0548006820440449C6
:1015500008600020034908800120F4E72F100020D4
:101560003C0000204000002010B5FFF7B7FF044604
:10157000A4F5806000F1006010BD00000348006920
:1015800040F08000014908617047000000200240DF
:1015900070B5044600F028F80546A5B10B4800696F
:1015A00040F002000949086108464461006940F0C2
:1015B0004000086100F018F805460448006920F072
:1015C000020002490861284670BD00000020024068
:1015D0000248034948600348486070472301674553
:1015E00000200240AB89EFCD4FF4F01000E0401E28
:1015F0000349C96801F0010109B10028F7D170471A
:101600000020024070B506460C4627E015480088C9
:10161000C0F5806085B2AC420DDA1349114A1288D8
:10162000881822463146FEF789FD0E48008820447E
:101630000C49088013E00C490A4A128888182A4687
:101640003146FEF77BFD4FF48060FFF771FF08B96C
:10165000002070BD2E44601B84B200BFD6E700BFDF
:101660000120F6E7400000202F1000200348044925
:10167000086000200349088070470000002000082F
:101680003C000020400000207CB504460D460F4879
:101690000088FFF74DFF08B900207CBD21460C48AB
:1016A000FFF724FFA84201D00020F6E7009401953F
:1016B000FFF75AFF064601230822694600F00AF8A0
:1016C00008B10120E9E70020E7E700004000002022
:1016D000002000082DE9F04706460C4617469846BC
:1016E00017B90120BDE8F087FFF772FFB8F1000FCE
:1016F00005D03046FFF74CFF08B90020F2E764251B
:1017000004EB070919E0FFF76FFF054605B916E07E
:101710000D48006940F001000B4908612068306005
:10172000FFF762FF05460848006920F001000649FE
:10173000086105B903E0361D241D4C45E3D300BF05
:10174000FFF71CFF2846CDE70020024000200021C3
:10175000264A126842F00102244B1A6000BF401C66
:10176000224A126802F0020111B9B0F5A06FF6D159
:101770001E4A126802F002020AB900BFFEE71B4AC5
:1017800052681A4B5A601A4652685A601A46526892
:1017900042F480625A601A465268154B1A40134B45
:1017A0005A601A465268134B1A43104B5A601A4635
:1017B000126842F080721A6000BF0C4A126802F090
:1017C0000072002AF9D0094A526822F00302074B3E
:1017D0005A601A46526842F002025A6000BF034A39
:1017E000526802F00802002AF9D070470010024047
:1017F000FFFFC3F7000028082DE9F04704460D4617
:101800000027B846B94600261D49601A8C421CD0F4
:1018100006DC1C48204470B1B0F5806F1FD10FE08A
:10182000B0F5806F16D0B0F56C4F18D10320FFF7DC
:1018300047F9074614E00220FFF742F907460FE098
:101840000220FFF73DF907460AE00220FFF738F9CA
:10185000074605E00220FFF733F9074600E000BF26
:1018600000BF07EB5500B0FBF5F64FF6F07006EA47
:10187000000806F00F0948EA0900A060BDE8F087FB
:10188000004C004000BCFFBF0A460021416921F026
:101890008001114341617047C16841F40051C1604A
:1018A00070470A460021416921F4007111434161EA
:1018B00070470A460021416921F48071114341615A
:1018C0007047C26822F4C062C260C2680A43C26044
:1018D00070470A460021C16821F004011143C1602C
:1018E0007047026922F44052026102690A430261B0
:1018F00070470A460021C16821F008011143C16008
:101900007047C26822F48052C260C2680A43C26053
:10191000704700003419000800000020600000003B
:10192000800200089419000860000020D0330000F5
:10193000900200080000000000000000000000000D
:101940000000000000000000000000000000000097
:1019500013000020060000000000000024100020FA
:101960000B0000000000000000000000000000006C
:101970000000000000001831421084BB1600000077
:10198000000000000B000000000000000003000049
:0419900000F36F06EB
:0C1FF000A09F00002159BB6EFFFFFFFF07
:10200000B832002019210008837600088572000884
:1020100077760008F12B0008A19500080000000069
:10202000000000000000000000000000DD85000846
:10203000FF27000800000000FD770008998D0008C8
:102040003321000833210008332100086579000896
:1020500033210008332100084D4C0008294D0008A9
:10206000332100083B4D00084D4D00083321000886
:1020700033210008332100083321000833210008F0
:10208000332100083321000833210008C1920008E1
:10209000899300083321000833210008754D00089A
:1020A00033210008332100083321000833210008C0
:1020B0003321000821910008332100083321000852
:1020C00033210008332100083321000833210008A0
:1020D000332100089191000829920008332100085B
:1020E0006D4C000833210008332100080000000077
:1020F00000000000000000000000000000000000E0
:1021000033210008DFF80CD000F048FB00480047FE
:10211000C9AB0008B832002006488047064800478F
:10212000FEE7FEE7FEE7FEE7FEE7FEE7FEE7FEE787
:10213000FEE7FEE7BD9000080521000840EA010324
:102140009B0703D009E008C9121F08C0042AFAD26D
:1021500003E011F8013B00F8013B521EF9D2704731
:10216000D2B201E000F8012B491EFBD270470022D9
:10217000F6E710B513460A4604461946FFF7F0FF86
:10218000204610BD421C10F8011B0029FBD1801A0B
:10219000704730B504460020034600E05B1C9342C4
:1021A00003D2E05CCD5C401BF8D030BD80EA010278
:1021B00010B502F00043400022D04A001FD0010EAB
:1021C00001EB1261C0F35600C2F3560240F4000066
:1021D00042F40002A0FB022000047F39140400D066
:1021E000401C50EA124001D44000491EC2B20C0605
:1021F00004EBD010401C4008802A02D003E00020ED
:1022000010BD20F00100002900DA0020184310BDA5
:102210002DE9FE4F804681EA0300C00F0C46009076
:1022200021F0004123F00045B8EB0200A94105D29E
:102230004046214690461C460B46024623F000408D
:10224000104347D0270DC7F30A00C3F30A51029089
:10225000401A019040286BDAC3F3130040F4801B4E
:102260000098924620B10023D2EB030A63EB0B0BDC
:1022700001985946C0F14002504600F0CAF906469E
:102280000D4650465946019A00F0E2F910EB08005D
:102290006141002487EA115284EAE7731A4340D06F
:1022A000009A62B3019A012A4FEA075215DC001B1B
:1022B00061EB02014FF0004202EA0752CDE9004211
:1022C000001C41F5801132462B4600F019FA03B08C
:1022D000BDE8F08F40462146F9E7001B61EB0201A3
:1022E000001C41F5801300185B412018A2F500176F
:1022F00047EB030140EAD570B6196D4111E06D0856
:102300004FEA360645EAC0754FEA0752001B61EBFB
:102310000201001C41F5801149084FEA3000001904
:10232000514132462B4603B0BDE8F04F00F0D9B919
:102330000098012240000023D0EB020263EBE0731F
:10234000009821464FEAE074B8EB000061EB04010D
:10235000E9E783F000435BE781F0004158E72DE9AE
:10236000FE4F81EA030404F0004421F00041009490
:102370004FF0000B23F0004350EA01045ED052EA14
:1023800003045BD0C3F30A54C1F30A552C44A4F2EE
:10239000F3340194A0FB0254C1F3130141F4801102
:1023A000C3F3130343F4801301FB024400FB034E09
:1023B000840A970A44EA815447EA8357A4FB0768D2
:1023C00002958D0A05FB07854FEA932C04FB0C54FC
:1023D0002705029D4FEA065847EA1637B5EB080570
:1023E0006EEB070C870E920E47EA811742EA8312C2
:1023F000A7FB0201B6EB0B0164EB00042B0D43EAD3
:102400000C335E1844EB1C50DA465146E7FB0201E0
:10241000C5F313044FEA0B3343EA14534FEA043273
:10242000019C43EA0603A4F10C040294009CCDE94C
:1024300000B400F065F903B0BDE8F08F002001465C
:10244000F9E72DE9F04D81EA030404F0004B21F097
:10245000004514464FF0000A23F0004150EA0502FF
:1024600020D054EA01021DD0C5F30A570246C5F335
:102470001303C1F31300C1F30A5640F4801543F46B
:102480008013A7EB0608101BD64608F2FD3873EB45
:10249000050002D308F1010801E092185B41B8F190
:1024A000000F03DA00200146BDE8F08D00204FF454
:1024B0008011064684460EE0171B73EB050705D313
:1024C000121B63EB050306434CEA010C49084FEA73
:1024D000300092185B4150EA0107EDD152EA030047
:1024E00012D082EA040083EA0501084305D0101BDC
:1024F000AB4106D20122002306E000224FF0004348
:1025000002E06FF0010253101AEB06004CEB085189
:1025100010EB0A0041EB0B01BDE8F04D00F0E1B813
:10252000C10F80EAE0700844CA079623002100F03A
:10253000AAB80EB540F2334102910021CDE9001155
:102540000A460B4600F0DCF803B000BD00F0004284
:1025500020F00040C10DC0F3160040F400007F29B8
:1025600001DA00207047962903DCC1F19601C840CA
:1025700001E096398840002AF4D040427047C1F308
:102580000A5210B5C1F3130140F2FF3341F4801138
:102590009A4201DA002010BD40F233439A42A2F27F
:1025A000334203DC524200F043F810BD904010BDAE
:1025B0002DE9F05F0546002092469B468846064678
:1025C000814640241BE0284641464746224600F00B
:1025D0002FF853465A46C01A914110D31146184657
:1025E000224600F016F82D1A67EB01084F462246E6
:1025F0000120002100F00DF817EB00094E41201ECC
:10260000A4F10104DFDC484631462A464346BDE8D2
:10261000F09F202A04DB203A00FA02F100207047E4
:102620009140C2F1200320FA03F319439040704710
:10263000202A04DB203A21FA02F00021704721FA17
:1026400002F3D040C2F1200291400843194670477E
:10265000202A06DBCB17203A41FA02F043EAE07366
:1026600006E041FA02F3D040C2F120029140084353
:10267000194670470029A8BF7047401C490008BF91
:1026800020F00100704710B4B0FA80FC00FA0CF0A2
:1026900050EA010404BF10BC704749B1CCF12004DA
:1026A00021FA04F411FA0CF118BF01212143084367
:1026B000A3EB0C01CB1D4FEA00614FEA102042BF93
:1026C000002010BC704700EBC35010440029A4BF89
:1026D00010BC7047401C490008BF20F0010010BC2E
:1026E000704710B5141E73F1000408DA401C41F164
:1026F000000192185B411A4301D120F0010010BD86
:102700002DE9F04D92469B4611B1B1FA81F202E0FB
:10271000B0FA80F220329046FFF77BFF04460F4666
:1027200040EA0A0041EA0B0153465A46084313D0D7
:10273000114653EA010019D0C8F140025046FFF794
:1027400077FF05460E46504659464246FFF761FF61
:10275000084305D0012004E020463946BDE8F08D4D
:102760000020054346EAE0762C4337430A98630588
:10277000E40AA0EB08000022FD0A44EA47540A30AC
:1027800002D500200146E9E7010510196941DDE99C
:10279000084500196941BDE8F04DA2E7064C074D18
:1027A00006E0E06840F0010394E807009847103421
:1027B000AC42F6D3FFF7AAFC88BE0008A8BE00080A
:1027C0000548007800B170470120034908700020D7
:1027D000488000BFF7E700003E00002010B500F081
:1027E000EFF800F02FFB00F0BDF900F075F810BD18
:1027F00010B5FFF7F3FF002000F098F810BD704708
:10280000505331303000000010B51348007808B341
:102810001148807800F00100A0B94FF480410F48C2
:1028200008F07AF9012804D100200B49087048808B
:1028300010E0002000F014F807484088401C0649CA
:10284000488007E0012000F00BF803484088401C56
:102850000149488010BD00003E00002000100140EA
:1028600010B504462CB101200749087000204880AB
:1028700008E005480021016000224FF400410348B0
:1028800008F0A2F810BD0000C400002000100140B4
:1028900010B50F480078D0B10D484088401C0C4955
:1028A000488008464088642808DB0122D103094893
:1028B00008F08AF806480021016008E004488078A2
:1028C00000F001024FF40041024808F07DF810BD0D
:1028D000C40000200010014010B540F2046008F070
:1028E0006FFD4FF44073032248210F4808F0BEF8F3
:1028F0000821022008F06EF802220021D00107F022
:1029000089FD4FF4807007F0E9FD0921022008F0ED
:1029100061F802220021100207F07CFD4FF40070E4
:1029200007F0DCFD10BD00000010014028B10121BE
:10293000044A1170C821518003E00021014A11703E
:10294000518070474600002000B50521034806F07D
:102950009DF9024880880249088000BD4A0900208C
:102960004C00002000B50521034806F08FF902480D
:1029700080880249088000BD540900204E000020D4
:1029800010B54FF0804009F047F8012000F0BEF983
:10299000074809F046F8074809F043F800210548C0
:1029A00008F0C9FF0120044908700449087010BDEF
:1029B00000040040002C01404A000020500000208C
:1029C00010B540F2036008F0FBFC00210A4808F053
:1029D000B3F84FF4406303221021084808F046F88A
:1029E0004FF48061054807F0EDFF4FF400610348A4
:1029F00007F0E8FF10BD000000021800000C0140C5
:102A0000505331303058585F5630315F30363032A5
:102A100031353434000000002DE9F05F4FF0000B39
:102A200036480078012801D0BDE8F09F4FF480714E
:102A3000334808F071F801281AD13248007801288B
:102A400016D1314808F073FF824640F6C410824523
:102A50000AD94FF0280B00202A490870274908702E
:102A6000294808F0D9FF2EE00220264908702AE004
:102A70004FF48071224808F04FF820BB21480078BD
:102A8000022820D1204808F052FF82464FEA5A0A15
:102A90005046FFF74EFD80464FF0C0421B4BFFF7FC
:102AA0005EFC064600221A4BFFF7CBFC0446FFF7FC
:102AB00066FD1FFA80FB0020124908700F4908705C
:102AC000114808F0A9FF0F480078A8B911480188FB
:102AD0000088401C0F4A10800F4820F811B01046A3
:102AE0000088052808DB0020114608800B48006894
:102AF00040F480200949086000BF95E7500000209D
:102B0000001001404A000020002C01408FC2D53F38
:102B100000002440420000204A090020000000205C
:102B200010B54FF0804008F077FF022000F0EEF87B
:102B3000084808F076FF084808F073FF00210648AF
:102B400008F0F9FE012005490870022004490870C8
:102B500010BD000000040040002C01404A0000208D
:102B6000500000201FB540F20B6008F029FC10480F
:102B700008F0E4FE684608F0E1FF6B20ADF80000C5
:102B80000020ADF80200ADF80400401E02900020C5
:102B9000ADF80C008DF80E006946054808F046FFB8
:102BA0000121034808F0B2FF014808F035FF1FBDBE
:102BB000002C014010B5024801F03CF910BD0000A6
:102BC0002006002010B5064800780649087006481F
:102BD000002101600548016004F05CFB10BD0000AD
:102BE000100000200F00002012000020160000201E
:102BF00000BFFEE700200149087070479C000020DC
:102C0000417070002DE9F05F4FF0000B36480078FE
:102C1000022801D0BDE8F09F4FF40071334807F05F
:102C20007BFF01281AD132480078012816D131489B
:102C300008F07DFE824640F6C41082450AD94FF066
:102C4000280B00202A49087027490870294808F0F5
:102C5000E3FE2EE00220264908702AE04FF40071BE
:102C6000224807F059FF20BB21480078022820D1D4
:102C7000204808F05CFE82464FEA5A0A5046FFF7A9
:102C800058FC80464FF0C0421B4BFFF768FB0646DE
:102C900000221A4BFFF7D5FB0446FFF770FC1FFA22
:102CA00080FB0020124908700F490870114808F095
:102CB000B3FE0F480078A8B9114801880088401C6D
:102CC0000F4A10800F4820F811B0104600880528E0
:102CD00008DB0020114608800B48006840F4002003
:102CE0000949086000BF95E750000020001001402E
:102CF0004A000020002C01408FC2D53F0000244034
:102D000044000020540900200000002070B588B065
:102D10000646012E02D0022E07D102E002246502EF
:102D200005E003244FF4006501E008B070BD00BF6A
:102D300040F2036008F044FB4FF4C06008F040FB31
:102D40002B46032218212A4807F090FE012129482A
:102D500007F0F2FE4FF4E06008F032FB4FF08040E5
:102D600008F0ECFD3520ADF804000020ADF80600B9
:102D7000ADF80800312003900020ADF810008DF868
:102D8000120001A94FF0804008F050FE0020ADF87D
:102D900018000120ADF814000020ADF81A00ADF8BD
:102DA0001600ADF81C00ADF81E0005AA21464FF034
:102DB000804008F059FC182221464FF0804008F06E
:102DC00076FD602221464FF0804008F043FD00224E
:102DD00021464FF0804008F07DFD4FF0804008F024
:102DE0003DFC4FF0804008F01CFE00BF9DE7000056
:102DF000000C01400002180010480078E0B10F48B4
:102E00004088401C0D49488008464088C82809DB96
:102E10000B48006840F480300949086000200749E9
:102E2000488009E005484088642805D104480068C6
:102E300040F400300249086070470000460000205E
:102E4000000000201FB540F2017008F0B9FA1348E5
:102E500008F074FD684608F071FE6B20ADF80000C4
:102E60000020ADF80200ADF804004FF4C8700290E5
:102E70000020ADF80C008DF80E006946074808F0F8
:102E8000D5FD0121054808F045FE044808F0C4FDC1
:102E9000002201211D2008F01BF81FBD0004004086
:102EA00070B507494868FFF73BFB05460549FFF742
:102EB0007DF90446FFF74AFB01498968081A70BD8D
:102EC00038070020CDCCCC3D70B507494868FFF7E6
:102ED00027FB05460549FFF769F90446FFF736FB6E
:102EE00001498968081A70BDB8080020CDCCCC3DD6
:102EF00010B5044604B910BD2078C0F340024FF469
:102F000000510A4807F060FD2078C0F3C0024FF47A
:102F10000041064807F058FD2078C0F300124FF436
:102F20008041024807F050FD00BFE4E7000C01407B
:102F300038B505460024052D77D2DFE805F0EF030C
:102F4000EEEDEC009DF8000020F0010000909DF8EF
:102F5000000020F0020000909DF8000020F0040026
:102F600000909DF8000020F0080000909DF80000FF
:102F700020F0100000906846FFF7BAFF00240DE033
:102F800004F05CFB4FF6E851884200D809E003F0FA
:102F900011FA0A2007F02CFA601C84B2B4F5FA7F0B
:102FA000EEDB00BFB4F5FA7F00DB20E2FE480078DC
:102FB000052876D2DFE800F0034B4C7C9400FB48F8
:102FC0000078032816D1002402E00A2007F010FA46
:102FD0002046611C8CB20F2803DAF54800780028DF
:102FE000F3D1F348007800B1DFE7002004F0B2FB32
:102FF00048B9DAE7ED480078012803D101F0FCF97F
:1030000008B1D2E7D1E7002402E00A2007F0F0F986
:103010002046611C8CB20F2803DAE64800780028AD
:10302000F3D1E448007808B1FBE3B3E3E248007869
:1030300038B9022004F03AFB00B9F2E3C82007F0E7
:10304000D7F9012004F032FB00B9EAE367E066E05B
:10305000002402E00A2007F0CBF92046611C8CB264
:103060000F2803DAD34800780028F3D1D14800783C
:1030700000B1D6E3012004F019FB00B9D1E300242C
:1030800002E00A2007F0B4F92046611C8CB20F2838
:1030900003DAC74800780028F3D1C548007808B1A2
:1030A000BFE337E0002004F055FB00B9B9E336E098
:1030B000002402E00A2007F09BF92046611C8CB234
:1030C0000F2803DABA4800780028F3D1B84800780E
:1030D00000B1A6E3002004F03DFB00B9A1E31EE02F
:1030E000B2480078032811D1002402E00A2007F03A
:1030F0007FF92046611C8CB20F2803DAAC480078B7
:103100000028F3D1002004F025FB02E0002004F0A9
:1031100021FB04E085E3CDE129E120E03BE300BFB2
:103120009DF8000020F0010000909DF8000020F0C4
:10313000020000909DF8000020F00400001D0090A7
:103140009DF8000020F00800083000909DF8000075
:1031500020F0100000906846FFF7CAFE58E39DF883
:10316000000020F0010000909DF8000020F0020017
:1031700000909DF8000020F0040000909DF80000F1
:1031800020F0080000909DF8000020F01000009052
:103190006846FFF7ADFE00240DE004F04FFA4FF64D
:1031A000E851884200D809E003F004F90A2007F04A
:1031B0001FF9601C84B2B4F5FA7FEEDB00BFB4F5F2
:1031C000FA7F00DB2DE378480078052874D2DFE829
:1031D00000F0034A7A7B930078480078032816D1E0
:1031E000002402E00A2007F003F92046611C8CB29B
:1031F0000F2803DA6F4800780028F3D16D48007873
:1032000000B10EE3002004F051FA48B909E36B481D
:103210000078012803D101F0D9F808B101E300E3F7
:10322000002402E00A2007F0E3F82046611C8CB27B
:103230000F2803DA5E4800780028F3D15C48007854
:1032400000B1EEE25C48007838B9022004F082FA5E
:1032500000B9E6E2C82007F0CBF8012004F07AFAC2
:1032600000B9DEE263E0002402E00A2007F0C0F8C3
:103270002046611C8CB20F2803DA4D4800780028E4
:10328000F3D14B48007800B1CBE2012004F062FAA0
:1032900000B9C6E2002402E00A2007F0A9F820469F
:1032A000611C8CB20F2803DA424800780028F3D161
:1032B0004048007808B1B4E238E0002004F0F6F9A4
:1032C00000B9AEE233E032E0002402E00A2007F069
:1032D0008FF82046611C8CB20F2803DA354800783D
:1032E0000028F3D13348007800B19AE2002004F0BE
:1032F000DDF900B995E21AE030480078032811D1D1
:10330000002402E00A2007F073F82046611C8CB20A
:103310000F2803DA274800780028F3D1002004F0B2
:10332000C5F902E0002004F0C1F900E079E200BF35
:103330009DF8000020F00100401C00909DF8000066
:1033400020F00200801C00909DF8000020F0040096
:1033500000909DF8000020F0080000909DF800000B
:1033600020F0100000906846FFF7C2FD50E29DF883
:10337000000020F0010000909DF8000020F0020005
:1033800000909DF8000020F0040000909DF80000DF
:1033900020F0080000909DF8000020F01000009040
:1033A0006846FFF7A5FD0BE0050000202E00002079
:1033B0002D000020280000201E00002029000020F1
:1033C00000240DE004F03AF94FF6E851884200D8A5
:1033D00009E002F0EFFF0A2007F00AF8601C84B24F
:1033E000B4F5FA7FEEDB00BFB4F5FA7F00DB18E23C
:1033F000FE48007805283AD2DFE800F003041C34C8
:1034000035000EE2002402E00A2006F0F1FF20461B
:10341000611C8CB20F2803DAF54800780028F3D13C
:10342000F348007800B1FCE1012004F093F900B901
:10343000F7E11DE0002402E00A2006F0D9FF204653
:10344000611C8CB20F2803DAEA4800780028F3D117
:10345000E848007800B1E4E1012004F027F900B960
:10346000DFE105E004E00A2006F0C2FF00E0D8E159
:1034700000BF9DF8000020F00100401C00909DF866
:10348000000020F00200801C00909DF8000020F059
:103490000400001D00909DF8000020F00800083096
:1034A00000909DF8000020F0100000906846FFF7A3
:1034B0001FFDADE19DF8000020F0010000909DF897
:1034C000000020F0020000909DF8000020F00400B1
:1034D00000909DF8000020F0080000909DF800008A
:1034E00020F0100000906846FFF702FD002004F075
:1034F00087F9BE48007805287BD2DFE800F0030496
:103500004689EF008DE10A2006F072FF9DF8000069
:1035100020F00100401C00909DF8000020F0020007
:1035200000909DF8000020F00400001D00909DF820
:10353000000020F0080000909DF8000020F010002E
:10354000103000906846FFF7D3FC002402E00A2008
:1035500006F04EFF2046611C8CB20F2803DAA44807
:1035600000780028F3D1A248007800B159E1022088
:1035700004F0F0F800B954E1C82006F039FF01204A
:1035800004F0E8F800B94CE1E0E00A2006F030FF72
:103590009DF8000020F00100401C00909DF8000004
:1035A00020F0020000909DF8000020F00400001DB3
:1035B00000909DF8000020F0080000909DF80000A9
:1035C00020F01000103000906846FFF791FC0024B6
:1035D00002E00A2006F00CFF2046611C8CB20F2886
:1035E00003DA844800780028F3D18248007808B1D3
:1035F00017E1AAE0022004F059F800B911E1C8204F
:1036000006F0F6FE012004F051F800B909E19DE052
:103610007948806879498968884248D2002402E064
:103620000A2006F0E5FE2046611C8CB20F2803DA62
:10363000704800780028F3D16E48007800B1F0E0BF
:10364000002004F033F800B9EBE0322006F0D0FEA1
:103650000A2006F0CDFE9DF8000020F00100401C7D
:1036600000909DF8000020F0020000909DF80000FE
:1036700020F00400001D00909DF8000020F00800DC
:1036800000909DF8000020F0100010300090684677
:10369000FFF72EFC022004F009F800B9C1E0C820B1
:1036A00006F0A6FE012004F001F8E0BBB9E000241A
:1036B00002E00A2006F09CFE2046611C8CB20F2816
:1036C00003DA4B4800780028F3D14948007800B16C
:1036D000A7E0002004F03EF808B9A2E034E0322070
:1036E00006F086FE0A2006F083FE9DF8000020F01A
:1036F0000100401C00909DF8000020F002000090A6
:103700009DF8000020F00400001D00909DF80000CE
:1037100020F0080000909DF8000020F0100010300C
:103720000090684600E00EE0FFF7E2FB022004F0A4
:1037300011F800B975E0C82006F05AFE012004F027
:1037400009F800B96DE001E000E06AE000BF0A207E
:1037500006F04EFE9DF8000020F00100401C009095
:103760009DF8000020F0020000909DF8000020F07D
:103770000400001D00909DF8000020F0080000905B
:103780009DF8000020F01000103000906846FFF710
:10379000AFFB3DE000BF0020FFF762F89DF800009E
:1037A00020F0010000909DF8000020F00200009041
:1037B0009DF8000020F0040000909DF8000020F02B
:1037C000080000909DF8000020F01000009068466E
:1037D000FFF78EFB002503F03DFEC0B10B2006492C
:1037E00081F8680000210448C16609E00500002056
:1037F0002D0000202800002038070020B8080020F5
:103800000B201B4981F8680000211948C16600BFE0
:1038100000BF18489DF8001001701748057068B285
:1038200038BD9DF8000020F0010000909DF80000D8
:1038300020F0020000909DF8000020F004000090AD
:103840009DF8000020F0080000909DF8000020F096
:10385000100000906846FFF74BFB06489DF80010EB
:1038600001700020044908700846007840B2D7E78C
:10387000B8080020040000200500002070B50446B0
:1038800005251748007808B9002070BD062C1AD20B
:10389000DFE804F003050A0F141A0020F5E700F032
:1038A000E5FC00B1012511E000F0E4FC00B10225C7
:1038B0000CE000F0E3FC00B1032507E000F00CFD94
:1038C00000B1042502E000BF0020DEE700BF052DA7
:1038D00001DB0020D9E72846FFF72AFBC0B2D4E776
:1038E0000D0000201848007848B317484088401C55
:1038F0001549488008464088B0F5967F09DB0846A0
:10390000002101601148006840F480500F490860B0
:1039100018E00D484088C82806D10C48006840F4DB
:1039200080500A4908600DE007484088642809D1A2
:103930000648006840F480500449086002E0002016
:10394000014948807047000060000020000000200E
:103950001848007848B317484088401C15494880EB
:1039600008464088B0F5967F09DB084600210160D3
:103970001148006840F400500F49086018E00D48F5
:103980004088C82806D10C48006840F400500A4915
:1039900008600DE007484088642809D1064800689F
:1039A00040F400500449086002E0002001494880CA
:1039B00070470000720000200000002010B554483D
:1039C00054490968016054485449096801605448E1
:1039D00054490968016054484D49486053484E496C
:1039E000486053484E494860524800210160416098
:1039F00001814FF480715048FEF7B9FB4E484D49A4
:103A0000486040F2197007F0DBFC40F2036007F0F9
:103A1000D7FC4FF4C06007F0D3FC4FF4807303224F
:103A20004821464807F022F84FF40073032218217A
:103A3000424807F01BF801214FF4EA1007F07CF828
:103A400040F2026007F0BCFC8023032210213C48B6
:103A500007F00CF800228021394806F0B5FF3949FB
:103A6000002006F075FC3849002006F071FC37484C
:103A700006F01CFA00203349087148718871C8713A
:103A80000872487208704870042088700220C8705C
:103A9000182048812D4806F0A7FA00202A494881BD
:103AA00088810120C8811B480068000C08801948E3
:103AB00000884880012088804FF6FF70C880002071
:103AC000088101200874084606F006FA01201E4904
:103AD000488112480068000C08801048008848801F
:103AE000084606F0F9F90220174948810D48006898
:103AF000000C08800B4800884880084606F0ECF966
:103B000000F0A8FB0221114806F003FB10BD0000E5
:103B10007C0E002090000020860E002094000020E3
:103B2000900E0020980000205E0B00205E0C00200C
:103B30005E0D00209A0E00205E0A0020000C01405D
:103B4000000801405E0E00206A0E00200064004064
:103B500010B540F2197007F033FC40F2036007F033
:103B60002FFC4FF4C06007F02BFC4FF4807303224E
:103B700048213B4806F07AFF4FF4007303221821D6
:103B8000374806F073FF01214FF4EA1006F0D4FF26
:103B900040F2026007F014FC802303221021314818
:103BA00006F064FF002280212E4806F00DFF2E490A
:103BB000002006F0CDFB2D49002006F0C9FB2C4863
:103BC00006F074F900202849087148718871C8719D
:103BD0000872487208704870042088700220C8700B
:103BE00018204881224806F0FFF900201F4948812B
:103BF00088810120C8811F480068000C08801D488A
:103C000000884880012088804FF6FF70C88000201F
:103C1000088101200874084606F05EF90120134966
:103C2000488115480068000C0880134800884880C7
:103C3000084606F051F902200C4948810F480068F7
:103C4000000C08800D4800884880084606F044F9BA
:103C500000F000FB0221064806F05BFA10BD0000F0
:103C6000000C0140000801405E0E00206A0E00209A
:103C70000064004090000020940000209800002084
:103C800010B505F0A3FD0348002101700020FFF7E7
:103C90004FF910BD040000202DE9FC5F4FF0000932
:103CA00003F0E2FE40B15D4840785D4908725D482E
:103CB0004078487200208872594800685849486026
:103CC000564890F87000A0B15448407888B1084632
:103CD000007A5249497888420BDD5148007A4F49B1
:103CE0004978401A00F0FF094D48807A48444C4911
:103CF00088724A4840784A4908724A4890F87000E9
:103D0000A0B14848407888B10846407A454949788A
:103D100088420BDD4248407A42494978401A00F017
:103D2000FF093F48807A48443D4988723D484078C1
:103D30003B494872394840783A49497808443849FB
:103D4000C872B9F1000F38D00846807A072834DBF2
:103D500008464068B0F52F7F2FD9887AFEF7E9FB37
:103D600005460E462E494868FEF7E3FB07462A46FD
:103D70003346FEF766FBCDE900014FF033322A4BA4
:103D8000DDE90001FEF7EBFA0746884624484FF0CC
:103D90006632264BD0E906512846FEF7E0FA824605
:103DA0003A464346FEF734FA1D4AC2E9060110219D
:103DB00002F1100004F05CFC00BF1949C87AFEF75C
:103DC000B8FB07461648D0E906532A463846FEF7A0
:103DD000C6FA82460022164BFEF733FBCDE90001FE
:103DE000FEF7CDFB0446C82C00D9C8240C490C733F
:103DF0000846007B48B10948C07C00F0400020B96B
:103E00000848C07C00F0400030B104480078054903
:103E10000978084402490873BDE8FC9F3807002070
:103E200098010020B80800203333D33F6666E63F90
:103E300000408F4070B50446666800258022294600
:103E40006D1C7254522229466D1C72541F48027810
:103E500029466D1C72540088021229466D1C72544A
:103E60001B48027829466D1C7254008802122946AC
:103E70006D1C7254E07820F018001830E070208833
:103E800020F47E7000F506702080B4F8010020F464
:103E9000FE7000F58470A4F80100A07820F03E00C8
:103EA000801CA070681EC11700EB5171C910491C1D
:103EB000628861F38A126280E07820F0E000E070AE
:103EC00025810E21204604F051FC70BD4C000020DD
:103ED0004E00002070B50446666800BF2D4880780B
:103EE0002D494978884200D00FE02A48C0782A49F5
:103EF000C978884200D008E0264880882649B1F871
:103F00000D10884200D000E070BD00BF224840780C
:103F1000204988702048C078C8701F48B0F80D004C
:103F200088800725E07820F018000830E0702088AD
:103F300020F47E7000F506702080B4F8010020F4B3
:103F4000FE7000F58470A4F80100A07820F03E0017
:103F5000801CA070681EC11700EB5171C910491C6C
:103F6000628861F38A126280E07820F0E000E070FD
:103F700025812A4607493046FEF7E0F80120074927
:103F80000870002048800021204604F0EFFB00BFAD
:103F9000BAE700005200002038070020600000202F
:103FA00070B50446666800BF2D4880782D49497871
:103FB000884200D00FE02A48C0782A49C978884250
:103FC00000D008E0264880882649B1F80D108842C4
:103FD00000D000E070BD00BF2248407820498870C2
:103FE0002048C078C8701F48B0F80D0088800725A9
:103FF000E07820F018000830E070208820F47E700F
:1040000000F506702080B4F8010020F4FE7000F581
:104010008470A4F80100A07820F03E00801CA070FD
:10402000681EC11700EB5171C910491C628861F309
:104030008A126280E07820F0E000E07025812A4654
:1040400007493046FEF77AF801200749087000203A
:1040500048800521204604F089FB00BFBAE7000034
:1040600064000020B80800207200002010B5FFF79F
:10407000A5FC4FF480713E48FEF779F83D480021D9
:104080000160416001813A483A4948604FF48071CB
:104090003948FEF76CF83948002101604160018120
:1040A0003548364948604FF480713548FEF75FF86F
:1040B0003448002101604160018131483149486044
:1040C0004FF480713048FEF752F83048002101600B
:1040D000416001812C482D49486040212C48FEF761
:1040E00046F82C4800210160416001812848294997
:1040F00048602948002101608180817143F281106C
:1041000025490880254800210160818043F2821002
:10411000224908802248002101608180817143F298
:1041200081201F4908801F4800210160818043F2DF
:1041300082201C4908801C480021016041600181E7
:104140004FF48540184908801848002101604160FB
:1041500001814FF485401549088015480021016010
:10416000416001814FF484401149088010BD000076
:10417000B8010020B8020020C2020020C2030020C3
:10418000CC030020CC040020D6040020D60500205B
:10419000E0050020200600205200002059000020E9
:1041A000640000206B0000202C090020360900204C
:1041B0004009002070B5044666680A222249234857
:1041C000FDF7E7FF00B970BD20481F490A6802608B
:1041D0004A684260098901810A25E07820F01800C8
:1041E0000830E070208820F47E7000F50670208092
:1041F000B4F8010020F4FE7000F58470A4F801000A
:10420000A07820F03E00801CA070681EC11700EB53
:104210005171C910491C628861F38A126280E0788A
:1042200020F0E000E07025812A4608493046FDF77D
:1042300085FF012006490870002048800A21204699
:1042400004F094FA00BFBEE7360900202C090020D4
:104250003A00002010B500220321132006F038FE9A
:1042600000220321142006F033FE10BD10B503F028
:10427000F7F810BD10B503F04FF910BD70B5134835
:10428000007808B9002070BD1148007820B11148AD
:10429000007808B10020F6E703F0E2F810B103F06F
:1042A0003BF908B90020EEE7FEF7FAFD0546FEF7F8
:1042B0000BFE0446A54201DB2E1B00E0661B642EAC
:1042C00001DC0120DFE70020DDE700000500002021
:1042D0000E0000200F00002070B51D480078012856
:1042E00005D01B480078022801D0002070BD194875
:1042F000007828B118480078012801D00020F5E79F
:104300001648007808B10020F0E702F0BDFF08B1C0
:104310000020EBE703F0A4F810B103F0FDF808B9B2
:104320000020E3E70E48007808B10020DEE7FEF742
:10433000B7FD0546FEF7C8FD04464BF2B030854296
:1043400001DD844201DC0020D0E70120CEE700003F
:10435000050000200E0000200F0000201F0000209C
:104360001A00002010B54FF4C06007F029F80022B1
:1043700001210A2006F0ACFD0421022006F02AFBF0
:1043800002220021102006F045F8102006F0A6F8C1
:1043900010BD000010B5002004F054FC00200749B7
:1043A000087007484078642806DB0648407864288F
:1043B00002DB01200449087010BD00001D00002030
:1043C00038070020B8080020E000002010B50024C5
:1043D0000848C07C00F0080050B903F02FF90446EB
:1043E000601C28B103488068A04201D2012010BDA2
:1043F0000020FCE7B808002010B500240848C07C65
:1044000000F0080050B903F019F90446601C28B107
:1044100003488068A04201D2012010BD0020FCE7C3
:10442000380700202DE9F04105272B48007840B1DE
:104430002A48007828B104F04DF907463846BDE80F
:10444000F08103F00DF8E8B103F066F8D0B124482C
:10445000C07C00F00600062806D00B20204981F819
:10446000680003211E48C1661E48C07C00F006009B
:1044700006280CD00B201B4981F86800032119483D
:10448000C16604E004F026F907463846D7E7144829
:10449000406844F62061884203DC12484068884244
:1044A00004DD04F017F907463846C8E7FEF7F8FCC4
:1044B0000546FEF709FD0446A54201DB2E1B00E080
:1044C000661B40F6C410864204DD04F003F907467B
:1044D0003846B4E73846B2E70E0000200F0000204F
:1044E00038070020B808002070B505263A48007843
:1044F00040B13A480078012804D004F0EBF80646B1
:10450000304670BD3648007820B104F0E3F8064626
:104510003046F6E702F0B8FE20B104F0DBF80646BC
:104520003046EEE702F09CFF20B302F0F5FF08B33F
:104530002C48C07C00F0060006280AD001202A4939
:10454000087004F0C7F80646002027490870304676
:10455000D7E72648C07C00F0060006280FD00120CF
:104560002349087004F0B6F8064600202049087078
:104570003046C6E704F0AEF806463046C1E7FEF71F
:104580008FFC0546FEF7A0FC04464AF2F87085420F
:1045900001DD844208DC1748007840B90120154944
:1045A00008700020488002E0124800210160114894
:1045B000007878B10F484088B0F57A6F0ADB0D4873
:1045C0000021016004F086F80646012004490870C5
:1045D000304696E7304694E70E0000200F0000209A
:1045E0001F000020380700201B000020B808002012
:1045F0001C0000201200002010B5052402F030FF3E
:1046000098B10B48C07C00F00600062800D00024BA
:104610000848C07C00F00A0040B10B20054981F831
:10462000680000210348C16600E00024204610BD58
:1046300038070020B808002010B5052402F06CFFF0
:1046400098B10B48C07C00F00600062800D000247A
:104650000848C07C00F00A0040B10B20054981F8F1
:10466000680000210348C16600E00024204610BD18
:10467000B80800203807002010B5052404F02AFBF4
:1046800010B104F05BFB00B910BD1A480078052892
:1046900018D2DFE800F003070B0F130004F01AF83C
:1046A000044610E0FFF7A8FF04460CE0FFF7C4FF44
:1046B000044608E0FFF7B6FE044604E0FFF714FFE7
:1046C000044600E0E0E700BF052C06DB0A4800785E
:1046D00010B9012003F094F8D6E734B90648007801
:1046E000012802D1002003F08BF82046FEF720FCC1
:1046F00000BFC9E7050000200D00002010B50D48DF
:104700000078B0B10C4805F0E1FB90B10122110333
:104710000A4806F059F9084805F0C8FBFFF718FAEF
:1047200000224FF48051054806F04EF9002004495C
:10473000087010BD0D00002000640040000801401A
:104740009C00002010B50548FFF7C4FB0448FFF7A4
:1047500027FC0448FFF72EFD10BD0000C203002017
:10476000CC040020D605002010B5504840786128C0
:1047700003DB4F484078612802DA00204D49087079
:1047800002F082FD00286ED04B48007828B300204C
:104790004A4908704A48007804280AD10320FFF7E4
:1047A0006DF8032822D101221103464806F00CF9C6
:1047B0001CE001221103434806F006F94048007846
:1047C000012803D03E48007802280FD13E480078E7
:1047D00060B901203C49087008E039480078042895
:1047E00004D001221103374806F0EEF84FF480514F
:1047F000344806F099F9002857D02C48C078B8B949
:104800002B48C078A0B93148007828B901202F4939
:104810000870002048800EE02C48408842F2107159
:10482000884208DB294800210160FFF7B3FD02E060
:1048300026480021016022480078032835D11B4812
:10484000C07888B11A48407B00F02000F8B11748C2
:10485000406817494968084441F28831884224DA9F
:10486000FFF798FD21E013E01148C07878B10F48B8
:10487000407B00F0200050B10C4840680C4949686A
:10488000084441F2883188420FDAFFF783FD0CE0DB
:1048900000224FF480510B4806F096F80648007845
:1048A00018B10B4800780549087010BD3807002082
:1048B000B8080020E00000200E0000200F000020BB
:1048C00005000020000C01401D000020D400002045
:1048D000100000200448007820B103484088401CA4
:1048E0000149488070470000D400002010B570488E
:1048F0000078A8B16E484088642811DB6C4800211C
:1049000001604FF480616B4806F006F908B9012098
:1049100000E000206849C97860F3C3016648C170AF
:1049200066484078B8B165484088B0F5FA6F12DB48
:1049300000206249487048804FF400615D4806F0ED
:10494000EBF808B9012000E000205B49C97860F36A
:10495000C7115948C1705A480078A8B158484088D2
:10496000642811DB5648002101604FF48051514802
:1049700006F0D2F808B9012000E000204E49C978BD
:1049800060F304114C48C1704E48007830B14D4876
:104990004088642802DB4B48002101604A480078C7
:1049A000A0B149484088642810DB474800210160D5
:1049B0004021464806F0B0F808B9012000E0002088
:1049C0003D49C97860F300013B48C1704048007818
:1049D000C0B13F484088642814DB00203C4948802F
:1049E0003C48007858B93C48006808B1012000E014
:1049F00000203149C97860F382012F48C17000203E
:104A00003549086035480078A0B1344840886428AA
:104A100010DB3248002101600121314806F07CF8AA
:104A200008B9012000E000202349097960F3000162
:104A30002148017102F028FC1F49097960F3410106
:104A40001D480171274840781B4948712548007866
:104A5000887125480078C871244800780872244875
:104A60000078487223480A6802604A6842600989EF
:104A700001811021154806F057F81E49C97860F3E6
:104A800041011C48C1700221104806F04DF8194937
:104A9000C97860F345111748C17001210B4806F031
:104AA00043F81449C97860F386111248C17010BDEB
:104AB000AC0000200010014036090020D800002082
:104AC000B0000020B4000020B8000020000C01401D
:104AD000BC000020D0000020DC000020C00000202E
:104AE0000014014036000020290000202E00002084
:104AF000050000204009002010B5094800680004A6
:104B00008209A2F5805000F100610B88088842F20A
:104B10002334A04201D1012010BD0020FCE7000099
:104B2000E0F7FF1F2DE9F0411A48006800048609EC
:104B3000A6F5006000F10064002543F2300720680C
:104B4000401C30B1122221461348FDF7F7FABDE8A8
:104B5000F08105F02BFE00F043FB204605F0B0FD90
:104B6000002507E000F03CFB6019394605F032FDF6
:104B7000A81CC5B2122DF5DB05F08CFDA6F5006072
:104B800000F10064122221460348FDF7D7FA00BF66
:104B9000DDE70000E0F7FF1FF800002010B503F08C
:104BA00011FD58B1104890F87000E0B901200E498D
:104BB00081F87000052081F8680014E00A4890F838
:104BC000700080B174210848FDF7D1FA0748002130
:104BD000016041608160002005490870052002499C
:104BE00081F8680000BF10BD380700202C070020A6
:104BF0002800002010B503F0EBFC58B1104890F8E5
:104C00007000E0B901200E4981F87000052081F89C
:104C1000680014E00A4890F8700080B174210848D8
:104C2000FDF7A5FA0748002101604160816000207E
:104C3000054908700520024981F8680000BF10BDD1
:104C4000B8080020AC0800202D00002010B501207D
:104C500005F04AFC38B1012005F040FC0120024972
:104C600008700020488010BDC000002010B54FF42F
:104C7000806005F039FC40B14FF4806005F02EFCF7
:104C8000012024490870002048804FF4006005F09E
:104C90002BFC58B14FF4006005F020FC1E48007852
:104CA00020B101201C494870002048804FF48050FA
:104CB00005F01AFC40B14FF4805005F00FFC0120C4
:104CC00016490870002048804FF4005005F00CFC95
:104CD00018B14FF4005005F001FC4FF4804005F08E
:104CE00003FC60B14FF4804005F0F8FB0C480078FD
:104CF00018B101200B49087010BDFDF761FD4FF49C
:104D0000004005F0F1FB18B14FF4004005F0E6FB60
:104D100000BFF1E7AC000020D8000020B000002068
:104D2000760000207800002010B5022005F0DCFBA2
:104D300010B1022005F0D2FB10BD10B5082005F01F
:104D4000D3FB10B1082005F0C9FB10BD10B5102031
:104D500005F0CAFB50B1102005F0C0FB102104483B
:104D600005F0DAFE10B9012003F06CFF10BD000061
:104D70000010014010B5202005F0B6FB10B1202036
:104D800005F0ACFB402005F0AFFB38B1402005F04A
:104D9000A5FB01201649087000204880802005F0FE
:104DA000A3FB70B1802005F099FB1248007828B968
:104DB00011480068401C1049086002E000200E49BC
:104DC00008604FF4807005F08FFB28B14FF48070BD
:104DD00005F084FBFDF720FE4FF4007005F084FB26
:104DE00028B14FF4007005F079FBFDF70BFF10BD03
:104DF000B8000020D0000020DC00002010B54FF4E7
:104E0000C06006F0DDFA00220121282006F060F8DB
:104E10000A21022005F0DEFD02220021500205F0E9
:104E2000F9FA4FF4806005F059FB0B21022005F0E0
:104E3000D1FD02220021900205F0ECFA4FF400604F
:104E400005F04CFB0C21022005F0C4FD02220021DC
:104E5000D00205F0DFFA4FF4805005F03FFB0E2141
:104E6000022005F0B7FD01220021900305F0D2FADF
:104E70004FF4804005F032FB00220121172006F09C
:104E800027F80621012005F0A5FD0222002140207F
:104E900005F0C0FA402005F021FB00220121062088
:104EA00006F016F80021032005F094FD02220021EF
:104EB000012005F0AFFA012005F010FB07210120C9
:104EC00005F088FD01220021802005F0A3FA802052
:104ED00005F004FB10BD000010B540F2046006F0C0
:104EE0006FFA4FF4004303221021494805F0BEFD3C
:104EF0000020FDF7B5FC4FF48043032248214448CD
:104F000005F0B4FD40F2056006F05AFA4FF4C060B7
:104F100006F056FA0121C80305F00EFE0123032214
:104F200048213C4805F0A2FDC02303221021384847
:104F300005F09CFD00224021354805F045FD00228A
:104F40008021334805F040FD40F2036006F038FA56
:104F500003231A461021304805F088FD0022012164
:104F60002D4805F031FD002202212B4805F02CFDD3
:104F70004FF4705303224821254805F077FD40F295
:104F8000036006F01DFA302303221021224805F0A9
:104F90006DFD00221021204805F016FD0022202181
:104FA0001D4805F011FDC023032248211A4805F0D1
:104FB0005DFDFFF723FF0120184908706420488039
:104FC00001201749087048704FF4FA6048800120AA
:104FD0001449087064204880012013490870642037
:104FE0004880012011490870642048800120104940
:104FF00008706420488001200E49087064204880B1
:105000000D48002101600D4801600D48016010BD90
:105010000010014000140140000C0140AC000020D1
:10502000D8000020B0000020B4000020B80000200C
:10503000BC000020C0000020C8000020CC000020E0
:10504000D000002028B10122044B1A701A4651806A
:1050500002E0024A0023136070470000A80000200D
:1050600028B10122044B1A701A46518002E0024A0C
:105070000023136070470000EC00002010B5FFF71C
:105080002BFF88210148FDF772F810BD10010020A8
:105090001848007848B317484088401C1549488094
:1050A00008464088B0F5967F09DB0846002101607C
:1050B0001148006840F480400F49086018E00D482E
:1050C0004088C82806D10C48006840F480400A494E
:1050D00008600DE007484088642809D10648006848
:1050E00040F480400449086002E000200149488003
:1050F000704700003A0000200000002006F070FA1F
:10510000234806F079FD234806F076FD224804F096
:10511000CDFE02F042FC00BF40F21C7006F050F9D8
:105120000021012005F03EFF03F0C8FF06F066FAFB
:1051300002F04EFA02F082FA044606F051FA44F602
:105140002060844223D91548844220D2012080F374
:10515000138800BF00BF00BF00BF00BF00BFBFF388
:105160004F8F00BF00BF00BF0D48006800F4E06033
:105170000C490843001D0A49086000BF00BF00BF7A
:10518000BFF34F8F00BF00BF00BF00BFFEE7C3E704
:10519000003801400044004000640040C0D40100D9
:1051A0000CED00E00000FA050B48007890B10A48C9
:1051B0004088401C80B20849488041F288318842CA
:1051C00008DB0548002101600448006840F4001035
:1051D00002490860704700007E00002000000020A7
:1051E00010B540F2073005F0E5F910BD10B540F2FA
:1051F000026006F0E5F840F2036006F0E1F840F2E4
:10520000046006F0DDF84FF4C06006F0D9F8012321
:1052100003224821224805F029FC062303224821C5
:105220001F4805F023FC4FF48053032210211D4832
:1052300005F01CFC012211031A4805F0C5FB0121F1
:10524000194805F079FC4FF4004303224821154822
:1052500005F00CFC082303221021144805F006FC7D
:1052600000220821114805F0AFFB1023032248213A
:105270000B4805F0FBFB4FF48053032210210B4831
:1052800005F0F4FBFFF76EF8042303221021074812
:1052900005F0ECFB01220421044805F095FB10BD4C
:1052A000001001400008014000023000000C0140E5
:1052B00010B504460B460CB103B10AB9002010BD6D
:1052C000002104E0188801449B1C901E82B2012A30
:1052D000F8DC002A01DD1878014402E088B200EB16
:1052E0001141080C0028F9D1C84320800120E6E7CD
:1052F00010B504460B460CB103B10AB9002010BD2D
:10530000002104E0188801449B1C901E82B2012AEF
:10531000F8DC002A01DD1878014402E088B200EBD5
:105320001141080C0028F9D1C84320800120E6E78C
:1053300070B5044600250CB9002070BD3048807857
:10534000C0F3440020B12E488078C0F3440000E050
:10535000202070B12A488078C0F344002849498849
:10536000C1F38411884204D12548008908B1244D35
:1053700034E024488078C0F3440020B1214880788C
:10538000C0F3440000E0202070B11E488078C0F3D4
:1053900044001C494988C1F38411884204D119484A
:1053A000008908B1174D19E017488078C0F3440010
:1053B00020B115488078C0F3440000E0202068B197
:1053C00011488078C0F344000F494988C1F3841123
:1053D000884203D10C48008900B10B4D0DB9002063
:1053E000ABE7286820602A8969686068FCF7A6FE38
:1053F00028892081284602F053FB20899DE7000080
:105400007C0E0020860E0020900E00200248C078FE
:1054100000F00100704700003609002070B5054615
:105420000C461DB108480088844201DA002070BD96
:105430000548028805492846FCF780FE0248048892
:1054400002F04CFB2046F2E7E6000020B4110020F9
:1054500070B505460C461DB108480088844201DA43
:10546000002070BD0548028805492846FCF766FE05
:105470000248048802F024FB2046F2E7A200002044
:10548000A40F002010B540F2073005F093F810BDCE
:1054900010B502460B460020002104E0545C044491
:1054A000E0B24C1CE1B29942F8DB10BD70B5044685
:1054B000264600BF0CB9002070BDB078012800D08E
:1054C0006FE0F5780020F07031782046FFF7E0FFBC
:1054D000A84200D065E0042570780D285CD2DFE892
:1054E00000F0070D223D52535455565758595A0053
:1054F0000122D1032C4805F067FA4FE0605D0128D6
:1055000005D101220821284805F05EFA0AE0605D15
:10551000022805D100220821234805F055FA01E0B0
:105520000020C9E73AE0605D012808D100220103AC
:105530001E4805F049FA01201D4908700DE0605D24
:10554000022808D10122C102184805F03DFA0020C6
:105550001749087001E00020AEE71FE0605D0128F8
:1055600005D101222021104805F02EFA0AE0605DE5
:10557000022805D1002220210B4805F025FA01E080
:10558000002099E70AE009E008E007E006E005E00E
:1055900004E003E002E001E000208DE700BF01200D
:1055A0008AE700BF002087E7000C014000080140A7
:1055B0000D00002070B5044634B94FF480711B48CB
:1055C000FFF746FFC5B209E0012C05D121021748BB
:1055D000FFF724FFC5B201E0002070BD144804703D
:1055E00012480078A84201D00020F6E70F48FFF7E4
:1055F0005DFF08B90020F0E70C4800F0B1F808B9E9
:105600000020EAE734B90948017803F00BF950B9F2
:105610000020E2E7012C06D10448017803F082F86B
:1056200008B90020D9E70120D7E700005E09002073
:105630007700002010B54FF40051364805F06CFAA1
:1056400018B1FFF759FA00B910BD334805F022FD33
:10565000002004F051F80120304908703048002142
:10566000016000BFFFF74AF800F0A4FE2D48007863
:1056700000F0010040B10020FFF79CFF29480068BE
:1056800020F00100274908602648007800F0040057
:1056900040B10120FFF78EFF2248006820F004008F
:1056A000204908601F48006800F4803038B1FDF7D9
:1056B00067F91C48006820F480301A4908601948CE
:1056C000006800F4003038B1FDF72AFA1548006888
:1056D00020F40030134908601248006800F480206C
:1056E00048B1FDF731F9FDF765FA0E48006820F47E
:1056F00080200C4908600B48006800F40020002856
:10570000B0D0FDF72FF90748006820F400200549C4
:105710000860A7E700100140443322117600002002
:1057200024000020000000200B48007890B10A48B7
:105730004088401C80B20849488040F6B831884211
:1057400008DD0548002101600448006840F480003D
:1057500002490860704700007A0000200000002025
:105760002DE9F04105462E4615B90020BDE8F0812F
:1057700070780D2877D2DFE800F0070D1319277A2B
:10578000F1F0EFEEEDECEB00042400222146641C66
:105790006A548CE3042400222146641C6A5486E384
:1057A000042400222146641C6A5480E3042440211E
:1057B000FA4805F0B1F908B1012200E000222046C4
:1057C000611CCCB22A5472E30424285D01280AD15A
:1057D00000220421F14805F0F7F800222046611C60
:1057E000CCB22A5442E0285D022810D10020EC49B6
:1057F00008700122D103EB4805F0E6F80121EA48E0
:1058000005F08AF92146621CD4B268542EE0285D66
:10581000032809D1E24802782046611CCCB22A5400
:105820000020DF49087021E0285D04280DD1002206
:105830004103DC4805F0C8F80121DB4805F06CF9AC
:105840002146621CD4B2685410E0285D05280BD1B3
:1058500001220421D14805F0B7F800222046611C3E
:10586000CCB22A5402E021E300207FE71FE30424A6
:10587000285D01283AD100224103C84805F0A4F868
:1058800000226103C54805F09FF800222103C348A8
:1058900005F09AF8642004F0ABFD0221C14805F040
:1058A0003BF92146621CD4B268540421BD4805F07E
:1058B00033F92146621CD4B2685401F0BFFE07469A
:1058C0002046611CCCB22F54C7F307222046611C2E
:1058D000CCB22A54C7F307422046611CCCB22A54EA
:1058E0003A0E2046611CCCB22A547EE1285D022883
:1058F00045D1601C285C01280AD10122C103A748B8
:1059000005F062F800222046611CCCB22A546CE1FA
:10591000601C285C022822D1642004F069FD01F09B
:105920008DFE07462046611CCCB22F54C7F30722D8
:105930002046611CCCB22A54C7F307422046611CA2
:10594000CCB22A543A0E2046611CCCB22A544CE107
:105950007FE268E241E20CE2EBE1A2E146E1601C99
:10596000285C0328C1D100224FF400418B4805F088
:105970002BF800222046611CCCB22A5435E1285D68
:1059800003282BD1642004F033FD0221854805F063
:10599000C3F82146621CD4B268540421814805F042
:1059A000BBF82146621CD4B2685401F047FE07469A
:1059B0002046611CCCB22F54C7F307222046611C3D
:1059C000CCB22A54C7F307422046611CCCB22A54F9
:1059D0003A0E2046611CCCB22A5406E1285D042808
:1059E0004BD1601C285C012812D1002204216B4895
:1059F00004F0EAFF0A2004F0FBFC0122510367488F
:105A000004F0E2FF00222046611CCCB22A54ECE0F4
:105A1000601C285C02281BD1642004F0E9FC01F022
:105A20000DFE07462046611CCCB22F54C7F3072257
:105A30002046611CCCB22A54C7F307422046611CA1
:105A4000CCB22A543A0E2046611CCCB22A54CCE087
:105A5000601C285C032891D1012204214F4804F0E6
:105A6000B3FF00224FF400514C4804F0ADFF002278
:105A70002046611CCCB22A54B7E0285D05282BD102
:105A8000642004F0B5FC0221464805F045F82146A3
:105A9000621CD4B268540421424805F03DF8214606
:105AA000621CD4B2685401F0C9FD07462046611C4F
:105AB000CCB22F54C7F307222046611CCCB22A5423
:105AC000C7F307422046611CCCB22A543A0E204646
:105AD000611CCCB22A5488E0285D06283ED1601CA7
:105AE000285C01280AD1012281032C4804F06CFFB4
:105AF00000222046611CCCB22A5476E0601C285C4F
:105B000002281BD1642004F073FC01F097FD0746C6
:105B10002046611CCCB22F54C7F307222046611CDB
:105B2000CCB22A54C7F307422046611CCCB22A5497
:105B30003A0E2046611CCCB22A5456E0601C285C08
:105B4000032852D100224FF48041144804F03CFF56
:105B500000222046611CCCB22A5446E0285D07286A
:105B600024D1002204210D4804F02EFF0A2004F065
:105B70003FFC01225103094804F026FF0122D10312
:105B8000064804F021FF01229103044804F01CFFA1
:105B900000222046611CCCB22A5426E0000C0140B1
:105BA000780000200010014000140140285D082802
:105BB0000AD10022C102C44804F006FF0022204698
:105BC000611CCCB22A5410E0285D09280BD10022B8
:105BD0004FF40041BC4804F0F7FE00222046611C4F
:105BE000CCB22A5401E00020C0E560E10424285D25
:105BF000012819D100228021B44804F0E5FE0022DA
:105C00000121B14804F0E0FE01224021AF4804F038
:105C1000DBFE01220221AC4804F0D6FE0022204621
:105C2000611CCCB22A543BE0285D022819D1002225
:105C30004021A64804F0C8FE00220221A24804F038
:105C4000C3FE01228021A14804F0BEFE01221146BC
:105C50009D4804F0B9FE00222046611CCCB22A54B3
:105C60001EE0285D032819D100228021974804F006
:105C7000ABFE00220121944804F0A6FE0022402140
:105C8000924804F0A1FE002202218F4804F09CFEFD
:105C900000222046611CCCB22A5401E0002065E5B8
:105CA00005E10424285D01281ED18102874804F003
:105CB00033FF2146621CD4B268544FF4006183481C
:105CC00004F02AFF08B1012200E000222046611CF6
:105CD000CCB22A544FF480517C4804F01DFF214679
:105CE000621CD4B2685423E0285D02281ED1410210
:105CF000764804F011FF2146621CD4B268544FF478
:105D00000061724804F008FF08B1012200E000229F
:105D10002046611CCCB22A544FF480516B4804F0E9
:105D2000FBFE2146621CD4B2685401E000201DE550
:105D3000BDE00424285D01280AD101221021624817
:105D400004F042FE00222146601CC4B26A540FE0F7
:105D5000285D02280AD1002210215B4804F034FE9D
:105D600000222046611CCCB22A5401E00020FDE450
:105D70009DE00424285D012814D1002054490860C6
:105D8000642004F035FB5248006828B10122204607
:105D9000611CCCB22A541FE000222046611CCCB208
:105DA0002A5419E0285D022814D1002048490860CF
:105DB000642004F01DFB4648006828B101222046FB
:105DC000611CCCB22A5407E000222146601CC4B2F8
:105DD0006A5401E00020C9E469E00424285D012838
:105DE0000DD101220103384804F0EEFD102137489F
:105DF00004F092FE2146621CD4B2685412E0285D81
:105E000002280DD10022C1022F4804F0DDFD10212F
:105E10002E4804F081FE2146621CD4B2685401E091
:105E20000020A3E443E00424285D01280ED104F0FF
:105E300069FD284802782046611CCCB22A542548C6
:105E400042782046611CCCB22A5401E000208DE447
:105E50002DE00424285D012807D1FCF767FD00220E
:105E60002046611CCCB22A541FE0285D02281AD1BA
:105E7000194802782046611CCCB22A541648008882
:105E800002122046611CCCB22A54144802782046E3
:105E9000611CCCB22A541148008802122046611CB1
:105EA000CCB22A5401E0002060E400E000BF00BF53
:105EB00034700020B070F07031782846FFF7E8FAAF
:105EC000F070012052E40000000C0140001001407D
:105ED000DC000020360000204C0000204E00002096
:105EE00018B503465C68586800880090BDF800004B
:105EF000B0F5A44F06D06FF4A441084418B17F2830
:105F000014D111E014E0A07810B1012808D103E009
:105F10000020FCF70BFD05E00120FCF707FD01E088
:105F2000002018BD00BF03E00020FAE70020F8E7DA
:105F300000BF0120F5E7000008B501464868008869
:105F40000090BDF8000043F20613C21A984210D028
:105F500007DCB0F5445F09D0A0F54450053868B9B6
:105F600005E0062A04D07B2A08D103E008E007E018
:105F700006E005E00020044A107008BD0020FCE7A0
:105F800000BF0120F9E700006000002008B50146CD
:105F9000486800880090BDF8000043F20623C21A4A
:105FA000984210D007DCB0F5485F09D0A0F5485002
:105FB000053868B905E0062A04D07B2A08D103E039
:105FC00008E007E006E005E00020044A107008BD84
:105FD0000020FCE700BF0120F9E70000720000206C
:105FE00070B5044660684578432D40D006DC312DFD
:105FF00009D0322D20D0422D6BD137E0482D34D03E
:10600000522D66D14CE03548216801602089334922
:1060100008810B461A8961685868FCF78FF82F4889
:10602000FFF78AFF08B9002070BD2C4801F004FE7C
:1060300008B90020F8E74DE029482168016020896F
:10604000274908810B461A8961685868FCF776F879
:106050002348FFF79BFF08B90020E5E7204801F03F
:10606000FBFE08B90020DFE734E000BF00BF1D4899
:106070002168016020891B4908810B461A896168E3
:106080005868FCF75BF8174800F030F808B90020B2
:10609000CAE7144801F0F0FF08B90020C4E719E08E
:1060A00011482168016020890F4908810B461A892F
:1060B00061685868FCF742F80B48FFF711FF08B910
:1060C0000020B1E7084801F017FD08B90020ABE750
:1060D00000E000BF00BF0120A6E70000C2030020CF
:1060E000CC040020D60500202006002038B5054647
:1060F0006C68686800880090BDF80000B0F5854FB6
:1061000074D00BDCA0F584400C2870D2DFE800F0DE
:106110003036373B4B4C4D515253545944F20232B6
:10612000811A90426BD014DC44F2F622A0EB0201FB
:1061300090426FD008DCA0F58040A0F53C700028AC
:1061400069D0052853D118E102296FD00B29F9D164
:1061500038E004296BD004DC01296AD00329F1D18D
:10616000C6E016297ED0A1F2FE410029EAD1FDE069
:10617000A07800F001008549087003E102E1A078F1
:1061800083490870FEE0A078012802D18149087097
:1061900008E0A078022803D100207E49087001E0C1
:1061A000002038BDEEE0EDE0ECE0A01C03F0D2FAF8
:1061B000E8E0E7E0E6E0E5E07748D4F802100160C7
:1061C000E0E0DFE0A07810B1012811D108E0002262
:1061D0002021724804F0F8FB00207149087009E0A2
:1061E000012220216D4804F0EFFB03E0BFE0C7E08F
:1061F0000020D6E700BF0A2004F0FAF8C2E0A07839
:1062000010B101280ED107E000221021634804F0EC
:10621000DBFB09E0B2E0AEE0012210215F4804F0B0
:10622000D3FB01E00020BCE700BFABE0A7E089E0C2
:10623000FFE7A07840B9002240215A4804F0C4FB8F
:106240000020594908704880A078012804D1012213
:106250004021544804F0B8FBA07802280BD1012259
:10626000402100E059E04F4804F0AEFB01204E49C8
:10627000087000204880A07803280AD1002240211D
:10628000484804F0A1FB0120474908704FF41670FC
:106290004880E07840B900228021424804F094FB15
:1062A0000020424908704880E078012804D101228A
:1062B00080213C4804F088FBE078022809D10122C3
:1062C0008021384804F080FB012038490870002004
:1062D0004880E07803280AD100228021314804F068
:1062E00073FB0120314908704FF41670488049E073
:1062F000A07810B101280CD105E000220221274826
:1063000004F062FB07E001220221244804F05CFB58
:1063100001E0002045E700BF34E0A07810B101287B
:106320000CD105E0002201211C4804F04DFB07E0E0
:1063300001221146194804F047FB01E0002030E734
:1063400000BF1FE0A07810B1012808D103E00020B1
:10635000FCF786FA05E00120FCF782FA01E0002054
:106360001FE700BF0A2004F043F80BE00AE000201A
:106370000F49087015E704F063FE00BF00BF01E09D
:1063800000200EE700BF01200BE70000D80000202E
:106390000E0000201000002098010020000C014099
:1063A0001F00002000100140C8000020CC00002089
:1063B0003A00002070B5B848FEF7BAFFC4B20CB975
:1063C000002070BDB548007801287DD1B448007820
:1063D000FF28FAD1B2484078FF28F6D1022421469E
:1063E000641CAF48405CAF4908700846007810282C
:1063F0006BD008DCA0F10A00062867D2DFE800F0C5
:10640000121CC5F4F3F214287ED006DC11287CD0CF
:1064100012287BD0132859D1B2E3302877D0312805
:10642000F9D1B5E39E49085DFCF782FD0546294692
:106430009DA003F007FAADE39E4801789EA003F00B
:1064400001FAA34890F87010A2A003F0FBF9A0484D
:1064500090F87110A5A003F0F5F99D480178A9A066
:1064600003F0F0F99A484178AAA003F0EBF99848B4
:106470008178ADA003F0E6F99548C178AEA003F0AD
:10648000E1F993484168B1A003F0DCF990488168D4
:10649000B3A003F0D7F98E48017BB7A003F0D2F97F
:1064A0008B48B0F80D10B8A003F0CCF98848D0F8AC
:1064B0000F10BAA003F0C6F98548C17CBDA003F057
:1064C000C1F91222824902E067E356E361E3153124
:1064D0007348FBF733FE002071498874BAA003F0BB
:1064E000B1F914227A4927316D48FBF727FE0020C5
:1064F0006B490875B7A003F0A5F97548B0F83B10D3
:10650000B8A003F09FF903E03BE337E337E33EE352
:106510006F48D0F83D10B7A003F094F96C48D0F85C
:106520004110B9A003F08EF96948D0F84510BCA01D
:1065300003F088F96648D0F84910BFA003F082F94B
:106540006348D0F84D10C3A003F07CF96048D0F840
:106550005110C7A003F076F95D48D0F85510C9A0D6
:1065600003F070F95A48D0F85910CCA003F06AF93A
:106570005748D0F85D10CFA003F064F95448D0F824
:106580006110D2A003F05EF904E3D6480178D6A0EA
:1065900003F058F9DA4890F87010DAA003F052F9D5
:1065A000D74890F87110DDA003F04CF9D448017879
:1065B000E0A003F047F9D2484178E2A003F042F9A5
:1065C000CF488178E4A003F03DF9CD48C178E6A03A
:1065D00003F038F9CA484168E8A003F033F9C84825
:1065E000816802E0B1E298E279E2E9A003F02AF9D9
:1065F000C348017BECA003F025F9C148B0F80D10A9
:10660000EDA003F01FF9BE48D0F80F10EFA003F083
:1066100019F9BB48C17CF3A003F014F91222B84960
:1066200015311F48FBF78AFD00201D498874F2A030
:1066300003F008F91422B24927311948FBF77EFD0F
:10664000002017490875EFA003F0FCF8AC48B0F83B
:106650003B10F0A003F0F6F8A948D0F83D10F1A0E7
:1066600003F0F0F8A648D0F84110F3A003F0EAF8E0
:10667000A348D0F84510F6A003F0E4F8A048D0F8FD
:106680004910F9A003F0DEF89D48D0F84D10FDA0A8
:1066900003F0D8F804E20000B80200202000002037
:1066A000B80100202100002072657475726E3A25D1
:1066B000640D0A00290000207375625F626D735FCC
:1066C000315F6C745F73746174653A25640D0A0000
:1066D0003807002072733438355F636F6E6E656300
:1066E000745F313A25640D0A00000000727334387B
:1066F000355F74696D655F6F75745F313A25640D40
:106700000A000000796A6B78736C635F313A256424
:106710000D0A00006D5F70657263656E745F313ADB
:1067200025640D0A00000000796A63647763736A68
:106730005F313A25640D0A006368617267655F66C0
:106740006C61675F313A25640D0A00006D5F637507
:106750007272656E745F313A25646D610D0A0000D6
:106760006D5F746F74616C5F766F6C5F313A257525
:106770006D760D0A00000000626D735F74656D70C8
:106780005F313A25640D0A00776F726B5F73746135
:106790007475735F313A25780D0A000062616E6C82
:1067A000616E63655F63656C6C5F313A25780D0AD5
:1067B00000000000626D735F7374617475735F3104
:1067C0003A25780D0A000000736E5F313A25730D8B
:1067D0000A000000736F66745F7665725F313A2558
:1067E000730D0A006463736D78735F313A25640D2D
:1067F0000A0000004368617267655F4E756D5F3126
:106800003A256C750D0A00004F7643685F766F6C11
:106810005F4E756D5F313A256C750D0A0000000002
:106820004F764469735F766F6C5F4E756D5F313A7A
:10683000256C750D0A0000004F764368617267652C
:106840005F6375725F4E756D5F313A256C750D0A29
:10685000000000004F764469736368617267655F8A
:106860006375725F4E756D5F313A256C750D0A0068
:1068700053686F72745F4E756D5F313A256C750D9C
:106880000A000000556454656D706543685F4E757D
:106890006D5F313A256C750D0A0000005564546532
:1068A0006D70654469735F4E756D5F313A256C7527
:1068B0000D0A00004F7654656D706543685F4E7534
:1068C0006D5F313A256C750D0A0000004F765465F6
:1068D0006D70654469735F4E756D5F313A256C75F7
:1068E0000D0A00002E0000207375625F626D735FF9
:1068F000325F6C745F73746174653A25640D0A00CD
:10690000B808002072733438355F636F6E6E65634C
:10691000745F323A25640D0A000000007273343847
:10692000355F74696D655F6F75745F323A25640D0C
:106930000A000000796A6B78736C635F323A2564F1
:106940000D0A00006D5F70657263656E745F323AA8
:1069500025640D0A00000000796A63647763736A36
:106960005F323A25640D0A006368617267655F668D
:106970006C61675F323A25640D0A00006D5F6375D4
:106980007272656E745F323A25646D610D0A0000A3
:106990006D5F746F74616C5F766F6C5F323A2575F2
:1069A0006D760D0A00000000626D735F74656D7096
:1069B0005F323A25640D0A00776F726B5F73746102
:1069C0007475735F323A25780D0A000062616E6C4F
:1069D000616E63655F63656C6C5F323A25780D0AA2
:1069E00000000000626D735F7374617475735F32D1
:1069F0003A25780D0A000000736E5F323A25730D58
:106A00000A000000736F66745F7665725F323A2524
:106A1000730D0A006463736D78735F323A25640DF9
:106A20000A0000004368617267655F4E756D5F32F2
:106A30003A256C750D0A00004F7643685F766F6CDF
:106A40005F4E756D5F323A256C750D0A00000000CF
:106A50004F764469735F766F6C5F4E756D5F323A47
:106A6000256C750D0A0000004F76436861726765FA
:106A70005F6375725F4E756D5F323A256C750D0AF6
:106A8000000000004F764469736368617267655F58
:106A90006375725F4E756D5F323A256C750D0A0035
:106AA0008648D0F8511086A002F0CCFE8348D0F87A
:106AB000551088A002F0C6FE8048D0F859108BA06F
:106AC00002F0C0FE7D48D0F85D108EA002F0BAFE44
:106AD0007A48D0F8611091A002F0B4FE5AE09548CF
:106AE00090F9001094A002F0ADFE924890F90110C8
:106AF00097A002F0A7FE00F0A1FD054629469AA046
:106B000002F0A0FE9D4801789DA002F09BFEA148E6
:106B10000178A1A002F096FE3CE0A548005D38B1E6
:106B20000B20A44981F868000321A248C16606E051
:106B30000B20A04981F8680000219E48C1669D484D
:106B4000C16E9DA002F07EFE24E09948005D38B140
:106B50000B205A4981F8680003215848C16606E0B5
:106B60000B20564981F8680000215448C1665348FB
:106B7000C16E94A002F066FE0CE00BE00AE009E0B2
:106B800008E09348017893A002F05CFE02E001E087
:106B900000E000BF00BF012013E4042290A184485C
:106BA000FBF7F7FA002854D104228FA18048001D7A
:106BB000FBF7EFFA30B90120854908708CA002F08C
:106BC00041FE44E008228EA17948001DFBF7E1FA5E
:106BD00030B904207E4908708CA002F033FE36E004
:106BE00006228FA17248001DFBF7D3FA30B90220AC
:106BF000774908708CA002F025FE28E005228EA1BE
:106C00006B48001DFBF7C5FA30B9032070490870C6
:106C10008BA002F017FE1AE006228DA16448001D29
:106C2000FBF7B7FA30B90020694908708AA002F072
:106C300009FE0CE005228CA15D48001DFBF7A9FAB6
:106C400018B98BA002F0FEFD01E00020A4E70120AE
:106C5000A2E75F480078022807D155480078FC2851
:106C600003D153484078FC281FD0594800780328A6
:106C700007D14F480078FE2803D14D484078FE28C0
:106C800013D053480078042807D149480078FD28DC
:106C900003D147484078FD2807D000204C490870B0
:106CA0007748FFF79DF9012076E71221744801F03B
:106CB0005DFD08B900206FE701206DE7B8080020EE
:106CC00053686F72745F4E756D5F323A256C750D47
:106CD0000A000000556454656D706543685F4E7529
:106CE0006D5F323A256C750D0A00000055645465DD
:106CF0006D70654469735F4E756D5F323A256C75D2
:106D00000D0A00004F7654656D706543685F4E75DF
:106D10006D5F323A256C750D0A0000004F765465A0
:106D20006D70654469735F4E756D5F323A256C75A1
:106D30000D0A0000360000206374725F74656D7088
:106D4000657261747572655B305D3A25640D0A0089
:106D50006374725F74656D70657261747572655B82
:106D6000315D3A25640D0A004261747465725F56A4
:106D70006F6C3A256C750D0A0000000004000020BD
:106D800063625F76616C5F6C6173743A25640D0AAF
:106D9000000000000500002063625F6F7065726193
:106DA00074655F73746174653A25640D0A000000B0
:106DB000B801002038070020424D535F313A256466
:106DC0000D0A0000424D535F323A25640D0A00005F
:106DD000200000206D6F64653A25640D0A000000F4
:106DE0006D6F64650000000074657374000000003E
:106DF0007465737420737563636573732100000099
:106E00006A69616F7A68756E000000006A69616F77
:106E10007A68756E20737563636573732100000073
:106E20007065697A686900007065697A68692073BD
:106E3000756363657373210063657368690000009F
:106E400063657368692073756363657373210000FC
:106E5000747569636875000074756963687520737B
:106E60007563636573732100636163687500000077
:106E700063616368752073756363657373210000D4
:106E8000B802002010B54FF480712148FEF7E0FAF7
:106E90001F49097888422ED00C221EA11C48FBF7FE
:106EA00078F930BB1F48007818BB012002F024FCA1
:106EB000012080F3138800BF00BF00BF00BF00BFE8
:106EC00000BFBFF34F8F00BF00BF00BF1648006870
:106ED00000F4E06015490843001D1349086000BF35
:106EE00000BF00BFBFF34F8F00BF00BF00BF00BF98
:106EF000FEE7002010BD06480078082805D90448A0
:106F000000F06CF808B90020F4E70120F2E7000077
:106F10002C0600207A68656E676A69636573686924
:106F200000000000760000200CED00E00000FA05F3
:106F300010B54FF480712148FEF770FA1F490978A7
:106F400088422ED00C221EA11C48FBF722F930BB30
:106F50001F48007818BB012002F0CEFB012080F30F
:106F6000138800BF00BF00BF00BF00BF00BFBFF35A
:106F70004F8F00BF00BF00BF1648006800F4E060FC
:106F800015490843001D1349086000BF00BF00BF3A
:106F9000BFF34F8F00BF00BF00BF00BFFEE7002060
:106FA00010BD06480078082805D9044800F0C0F84C
:106FB00008B90020F4E70120F2E70000AC07002048
:106FC0007A68656E676A69636573686900000000C6
:106FD000760000200CED00E00000FA052DE9F041FC
:106FE00007463D4600BF687849490978884204D180
:106FF000A879162801D1E87900B986E04548002132
:107000000160416081604448006820F00800424906
:107010000860424C002084F871000120404908704B
:10702000002040490870204690F8700018B10320F5
:107030003D49087002E002203B490870AE880020FC
:10704000A8802A783946281DFEF732F98046B8F123
:10705000010F02D1A888B04200D056E00826B91925
:1070600015222046FBF76AF81536207D00F0010056
:1070700000B94AE0207D0009102827D2DFE800F09F
:1070800008090A0B0C0D1721232626222626242563
:107090001DE01CE01BE01AE019E0B919262204F1FA
:1070A0001500FBF74BF806F1260086B20FE0B91980
:1070B0002A2204F13B00FBF741F806F12A0086B2D0
:1070C00005E004E003E002E001E000E000BF00BFF3
:1070D00094F86800217DB0EB111F13D10020A06649
:1070E000E06612480078401CC0B2104908701E28A3
:1070F00005DD062084F868000020087002E000200A
:1071000084F868000120BDE8F08100BF0020FAE7A4
:10711000220000202C07002000000020380700205B
:107120002A00002028000020290000202B00002039
:107130002DE9F04107463D4600BF68784949097886
:10714000884204D1A879162801D1E87900B986E0EF
:10715000454800210160416081604448006820F09A
:10716000100042490860424C002084F87100012060
:1071700040490870002040490870204690F870008F
:1071800018B103203D49087002E002203B49087015
:10719000AE880020A8802A783946281DFEF7A8F876
:1071A0008046B8F1010F02D1A888B04200D056E065
:1071B0000826B91915222046FAF7C0FF1536207D9A
:1071C00000F0010000B94AE0207D0009102827D214
:1071D000DFE800F008090A0B0C0D172123262622F0
:1071E000262624251DE01CE01BE01AE019E0B91951
:1071F000262204F11500FAF7A1FF06F1260086B257
:107200000FE0B9192A2204F13B00FAF797FF06F1C3
:107210002A0086B205E004E003E002E001E000E0BD
:1072200000BF00BF94F86800217DB0EB111F13D19F
:107230000020A066E06612480078401CC0B21049E9
:1072400008701E2805DD062084F8680000200870FC
:1072500002E0002084F868000120BDE8F08100BF52
:107260000020FAE72C000020AC08002000000020DD
:10727000B80800202F0000202D0000202E00002044
:107280003000002000BFFEE7014800797047000091
:10729000A41000202DE9F04112480068000486097E
:1072A000A6F5406000F10064254620210E48FAF75B
:1072B0005EFF288840F2253188420CD008460A49F2
:1072C0000882002209490848C0E90621102110302F
:1072D00001F0CEF904E0044895E88E0010308EC02D
:1072E000BDE8F081E0F7FF1F9801002000C0824058
:1072F00070B55148007800287ED05048007850B9C9
:107300004F480078032800D170BD0320FCF7B6FA7F
:1073100003280BD1F8E74A480078042800D1F3E7A6
:107320000420FCF7ABFA042800D1EDE744480078CC
:1073300000287CD0012804D002283BD0042875D135
:1073400076E04FF480513F4803F0EEFBD8B13E4861
:10735000C07C00F01000102803D10220FCF78EFA48
:1073600027E03A480078012823D1FBF7ADFD044619
:10737000FBF796FD844202DA0220FCF77FFA022036
:107380003249087015E030484468002C01DB204683
:1073900000E06042B0F57A7F0BDCFBF795FD054617
:1073A000FBF77EFD00F5FA70854202DD0220FCF756
:1073B00065FA3EE04FF48051224803F0B5FBE0B19E
:1073C0002348C07C00F01000102803D10120FCF7F6
:1073D00055FA28E01D480078012824D1FBF760FD0C
:1073E0000446FBF771FD844202DA0120FCF746FAFD
:1073F00002201649087016E01CE015484468002C6D
:1074000001DB204600E06042B0F57A7F0BDCFBF741
:1074100047FD0546FBF758FD00F5FA70854202DD91
:107420000120FCF72BFA04E001E0FFE700BF00BFFA
:1074300000BF00BF00BF67E70E0000200F00002064
:1074400005000020000C0140380700201D0000202E
:10745000B80800200148C078C009704736090020EC
:1074600010B52648B0F80D4024F0100424F0200494
:1074700024F0800424F004044FF48051204803F0E9
:1074800053FB40B124F0020424F4006424F40054BB
:1074900024F4004405E024F0010424F4804424F49E
:1074A000805400BF17484078012800D122E01648D8
:1074B000007800B11EE015480078042809D10421A5
:1074C000134803F029FB08B9012000E0002000B9AF
:1074D00010E0FFF7BFFF00B10CE001F073F800B956
:1074E00008E004B106E00B480078032800D001E072
:1074F000012010BD00BF0020FBE70000380700207E
:10750000000C0140100100201B000020050000209D
:10751000001001402900002010B52648B0F80D40A9
:1075200024F0100424F0200424F0800424F0040447
:107530004FF48051204803F0F7FA40B124F00204E0
:1075400024F4006424F4005424F4004405E024F0FE
:10755000010424F4804424F4805400BF1748407888
:10756000022800D122E01648007800B11EE015483C
:107570000078042809D10221134803F0CDFA08B994
:10758000012000E0002000B910E0FFF763FF00B128
:107590000CE001F01DF800B908E004B106E00B486A
:1075A0000078032800D001E0012010BD00BF0020BA
:1075B000FBE70000B8080020000C0140100100208B
:1075C0001C00002005000020001001402E000020BB
:1075D00010B540F2026003F0F3FE4FF4C06003F018
:1075E000EFFE40F2096003F0EBFE032003F08CFD98
:1075F000202303220021024803F038FA10BD0000C6
:107600000008014000B501F027FB00BD10B502F0F5
:10761000EDF8012007490870002048800648002145
:107620000180002403E003F06DF9601CC4B2022C59
:10763000F9D310BD320000203600002038B50020FC
:107640000090441E6946052002F037FB012800D057
:107650000BE0BDF8000040F6E44148436521484393
:1076600040F6FF71B0FBF1F400BF204638BD10B505
:1076700002F0DEF810BD00BFFEE710B5FDF7B6FD65
:1076800010BD704710B5002807DA0A07140E054A26
:1076900000F00F031B1FD45403E00A07130E024A25
:1076A000135410BD18ED00E000E400E02DE9F041B6
:1076B00005464FF096080B20244981F8680035B143
:1076C000012D02D0022D08D103E0032407E000249D
:1076D00005E004244FF4FA6801E0002400BF00BF75
:1076E0001A48C4661A48006820F00100184908606A
:1076F00001F0D8F86006040E002700261CE00A20DE
:1077000002F076FE1248007800F0010090B11048B7
:10771000006820F001000E490860FFF7B3FB022D5E
:1077200006D00A48C07C2040A04202D1012700E0D8
:10773000012706E0701C86B20A2098FBF0F0B042E8
:10774000DDDC00BF78B2BDE8F08100003807002022
:10775000000000202DE9F04105464FF096080B206F
:10776000244981F8680035B1012D02D0022D08D1DD
:1077700003E0032407E0002405E004244FF4FA6842
:1077800001E0002400BF00BF1A48C4661A48006820
:1077900020F004001849086001F058F96006040E52
:1077A000002700261CE00A2002F022FE1248007882
:1077B00000F0040090B11048006820F004000E4969
:1077C0000860FFF7B5FB022D06D00A48C07C2040B8
:1077D000A04202D1012700E0012706E0701C86B21A
:1077E0000A2098FBF0F0B042DDDC00BF78B2BDE8C3
:1077F000F0810000B8080020000000207047000061
:1078000010B50446C4B1002204211C4803F0DCF882
:107810000120FBF725F800224FF48051184803F0AF
:10782000D3F801220821154803F0CEF800201549AD
:10783000087000F03DF91DE0012204210F4803F01B
:10784000C3F80020FBF70CF8012211030C4803F0E9
:10785000BBF8FBF7CFF900222021084803F0B4F869
:107860000020FBF763F800220821044803F0ACF87D
:1078700001F0F2F90448047010BD0000000C014052
:10788000000801401E0000200D00002010B5174820
:1078900090F8700018B104201549087002E001202A
:1078A00013490870114890F8710000B110BD1521FE
:1078B0000E48FAF75CFC26210C481530FAF757FC05
:1078C0002A210A483B30FAF752FC08480021816619
:1078D000C1660120054981F87100052081F8680022
:1078E00000200449087000BFE0E7000038070020CE
:1078F000290000202A00002010B5174890F87000D9
:1079000018B104201549087002E0012013490870DD
:10791000114890F8710000B110BD15210E48FAF71A
:1079200026FC26210C481530FAF721FC2A210A48AA
:107930003B30FAF71CFC084800218166C166012033
:10794000054981F87100052081F86800002004498C
:10795000087000BFE0E70000B80800202E000020FB
:107960002F00002010B5012003F0A2FD10B101206E
:1079700003F096FD022003F09BFD68B1022003F0A6
:107980008FFD4FF4003002F0A9FD03F0A5FD0020AB
:1079900003F076FD03F0A0FD10BD10B5002201211B
:1079A000032003F095FA40F21B7003F009FD40F24A
:1079B0001C7003F005FD03F0EBFA02F071FA0022EF
:1079C00011464FF4003002F025FD4FF4003002F074
:1079D00085FD4FF4003002F079FD4FF4106003F0A4
:1079E0006FFC4FF4106003F07BFC4FF4007003F069
:1079F00017FD40F60F0003F0E3FC03F087FD03F0F2
:107A00006BFD022003F060FD03F066FD282003F00B
:107A10006DFD03F061FD03F05FFD4FF47A7003F03C
:107A20000BFD03F059FD10BD10B51021014800F009
:107A30009DFE10BD2006002010B50321014800F076
:107A400095FE10BDC203002010B50821014800F0CA
:107A50008DFE10BDCC04002010B50C21014800F0B3
:107A600085FE10BDD605002010B5FDF7CFFC08B986
:107A7000012010BD0948006808494968884201D2C0
:107A80000120F6E70548807A28B10448406832288A
:107A900001D80120EDE70020EBE70000980100206D
:107AA00000B9704700210160018100BFF9E70000C3
:107AB0000020024908704880704700007E000020C6
:107AC00010B54FF480710348FAF751FB00200249CA
:107AD000088010BDA40F0020A200002010B54FF4B4
:107AE00080710348FAF743FB00200249088010BD6B
:107AF000B4110020E6000020F8B50446666860680E
:107B000000880090BDF80000B0F5A44F07D06FF4D6
:107B1000A4410844002830D07F284AD147E0E078CB
:107B2000C0F3C100012801D00120F8BD00250022CA
:107B300029466D1C7254522229466D1C7254002233
:107B400029466D1C72543848027829466D1C7254BF
:107B50003648027829466D1C725400880212294664
:107B60006D1C72543248027829466D1C725400888C
:107B7000021229466D1C72541DE0E078C0F3C1006A
:107B8000012801D00120D0E70025012229466D1CE3
:107B90007254522229466D1C7254002229466D1CD3
:107BA00072542148027829466D1C725403E000206B
:107BB000BBE70020B9E700BFE07820F018001030E4
:107BC000E070B4F801008108208861F3C9002080CA
:107BD000B4F8010020F4FE7000F58470A4F80100F0
:107BE000A07820F03E00801CA070681EC11700EB3A
:107BF0005171C910491C628861F38A126280E07871
:107C000020F0E000E07025810F21204600F0AEFD5D
:107C100038B90848006840F4006006490860002050
:107C200083E7012081E70000460000204C0000208F
:107C30004E00002000000020F8B504466668606829
:107C400000880090BDF8000043F20C12811A9042A7
:107C500057D009DCB0F5445F0DD0A0F5445005388D
:107C6000B8B301287CD163E001297CD0022979D006
:107C70007529F7D1ACE0E078C0F3C100012802D14A
:107C80007148007808B10120F8BD0225002229467C
:107C90006D1C7254701914226C49FAF74FFA6C4833
:107CA000007B90B16A48C07A68494978884203D11C
:107CB0006748007BF07008E06548007B63494978BD
:107CC0004843642190FBF1F0F07005F1140085B297
:107CD00082E0FFE7E078C0F3C100012802D15A48F2
:107CE000007808B10120CFE70225002229466D1C4B
:107CF00072547019122255491531FAF71FFA1235CC
:107D00006AE0E078C0F3C100012802D14E48007853
:107D100008B10120B8E70225002229466D1C7254E3
:107D20007019142249492731FAF708FA143553E03B
:107D3000E078C0F3C100012802D14348007808B1BF
:107D40000120A1E70225002229466D1C72543F4FF5
:107D50003B3770190E223946FAF7F0F90E353BE041
:107D600038E000E018E0E078C0F3C100012802D15B
:107D70003548007808B1012086E70225002229460F
:107D80006D1C7254314F3B377019102207F10E01F0
:107D9000FAF7D4F910351FE0E078C0F3C1000128EC
:107DA00002D12948007808B101206DE702250022A0
:107DB00029466D1C7254254F3B37701957F81E1F0A
:107DC000016079684160B9681E3F81600C3503E04D
:107DD000002059E7002057E700BFE07820F01800A6
:107DE0001030E070B4F801008108208861F3C90008
:107DF0002080B4F8010020F4FE7000F58470A4F82F
:107E00000100A07820F03E00801CA070681EC11701
:107E100000EB5171C910491C628861F38A126280BB
:107E2000E07820F0E000E07025810221204600F09B
:107E30009DFC38B90748006840F480700549086027
:107E4000002021E701201FE7600000203807002004
:107E50009801002000000020F8B5044666686068BC
:107E600000880090BDF8000043F20C22811A904275
:107E700057D009DCB0F5485F0DD0A0F54850053863
:107E8000B8B301287CD163E001297CD0022979D0E4
:107E90007529F7D1ACE0E078C0F3C100012802D128
:107EA0007148007808B10120F8BD0225002229465A
:107EB0006D1C7254701914226C49FAF73FF96C4822
:107EC000007B90B16A48C07A68494978884203D1FA
:107ED0006748007BF07008E06548007B634949789B
:107EE0004843642190FBF1F0F07005F1140085B275
:107EF00082E0FFE7E078C0F3C100012802D15A48D0
:107F0000007808B10120CFE70225002229466D1C28
:107F100072547019122255491531FAF70FF91235BA
:107F20006AE0E078C0F3C100012802D14E48007831
:107F300008B10120B8E70225002229466D1C7254C1
:107F40007019142249492731FAF7F8F8143553E02B
:107F5000E078C0F3C100012802D14348007808B19D
:107F60000120A1E70225002229466D1C72543F4FD3
:107F70003B3770190E223946FAF7E0F80E353BE030
:107F800038E000E018E0E078C0F3C100012802D139
:107F90003548007808B1012086E7022500222946ED
:107FA0006D1C7254314F3B377019102207F10E01CE
:107FB000FAF7C4F810351FE0E078C0F3C1000128DB
:107FC00002D12948007808B101206DE7022500227E
:107FD00029466D1C7254254F3B37701957F81E1FE8
:107FE000016079684160B9681E3F81600C3503E02B
:107FF000002059E7002057E700BFE07820F0180084
:108000001030E070B4F801008108208861F3C900E5
:108010002080B4F8010020F4FE7000F58470A4F80C
:108020000100A07820F03E00801CA070681EC117DF
:1080300000EB5171C910491C628861F38A12628099
:10804000E07820F0E000E07025810721204600F074
:108050008DFB38B90748006840F400700549086096
:10806000002021E701201FE772000020B80800204F
:1080700098010020000000202DE9F84306467568AD
:108080004FF00008706800880090BDF8000044F2CE
:108090000B22811A90426FD00BDCA0F584400B2894
:1080A0006BD2DFE800F0263D778D9EB4CADAF0EFA0
:1080B000EE00F72978D00CDCEB2976D004DC7529AA
:1080C00074D0EA2959D137E2ED2970D0F629F9D1D7
:1080D00073E1FB296CD004DCF8296AD0FA29F1D1CC
:1080E000BAE1A1F20D11002974D0B1F59D6FE9D16B
:1080F000F1E1F078C0F3C100012802D1FB4800781B
:1081000010B10120BDE8F8834FF48440F84908809D
:10811000002088700A2422462846FAF70FF817E252
:10812000F078C0F3C100012802D1F048007808B10E
:108130000120E7E70224EF48007848B100222046FA
:10814000611C8CB22A542046611C8CB22A5420E057
:10815000285D002812DD285D05280FDA285DE64934
:108160000978884202D0285DFBF788FB0022204670
:10817000611C8CB22A5406E016E1E7E10122204698
:10818000611C8CB22A54DC4802782046611C8CB2F7
:108190002A54DDE1F078C0F3C100012802D1D348B0
:1081A000007838B10120ADE72FE1C6E1C2E1C8E1B6
:1081B00072E141E1022400222146641C6A54C7E1B5
:1081C000F078C0F3C100012802D1C848007810B18E
:1081D000012097E750E1022400222146641C6A54E2
:1081E000B6E1F078C0F3C100012802D1BF480078A1
:1081F00008B1012086E7022400222146641C6A544B
:1082000028191422BD49F9F799FF1434A0E1F07838
:10821000C0F3C100012802D1B448007808B10120A0
:1082200070E7022400222146641C6A542819122295
:10823000B349F9F783FF12348AE1F078C0F3C10043
:10824000012802D1A948007808B101205AE7022488
:1082500000222146641C6A547AE14FF00008AC7891
:10826000012C01D0022C2CD1012C01D1022700E0DD
:1082700001273846FBF702FBB84205D04FF0020851
:1082800021E080E075E024E0012C04D1012001F020
:10829000FBF8C7B203E0012001F03CF9C7B26FB1AF
:1082A000012098490870A878487028794880E878B3
:1082B000897840EA01209349488004E04FF00308A0
:1082C00001E04FF0010802242146641C05F80180FA
:1082D0003EE14FF00008EC78A87840EA0424894891
:1082E0004088A0423DDB6C79287940EA0424802C48
:1082F00034D8022083490870E8788880A878097902
:1083000040EA01207F4988806879C8802879897986
:1083100040EA01207B49C8800846C288A91D083070
:10832000F9F70CFF77484078012804D1022001F0CA
:10833000ABF8C7B203E0022001F0ECF8C7B257B1C6
:10834000704880886F49498888420CD188216D48DF
:10835000F9F70DFF07E04FF0030804E04FF00208C3
:1083600001E04FF0010802242146641C05F8018059
:10837000EEE088216348F9F7FAFE02240022214644
:10838000641C6A54E4E0F078C0F3C100012802D113
:108390005648007808B10120B4E602245A48027B0E
:1083A0002146641C6A54D3E0012001F0A5F902249F
:1083B00000222146641C6A54CAE0F078C0F3C10070
:1083C000012802D14948007808B101209AE6022428
:1083D00000222146641C6A5440214C4802F09CFB58
:1083E00008B9012200E000222046611C8CB22A5408
:1083F0006420474948800120464908700020488091
:108400004549488045490860A2E0F078C0F3C100C2
:10841000012802D13548007808B1012072E6022413
:1084200000222146641C6A541021384802F07CFB6B
:108430002246641CA8548BE0F078C0F3C1000128E8
:1084400002D12A48007808B101205BE6022400220C
:108450002146641C6A547BE0F078C0F3C100012817
:1084600002D12248007808B101204BE60224002204
:108470002146641C6A546BE0F078C0F3C100012807
:1084800002D11A48007808B101203BE602240022FC
:108490002146641C6A545BE0F078C0F3C1000128F7
:1084A00002D11248007808B101202BE602240022F4
:1084B0002146641C6A540121194802F02DFB08B9B9
:1084C000012200E000222046611C8CB22A54642064
:1084D000144948803CE0F078C0F3C100012802D183
:1084E0000248007808B101200CE61DE03A000020A7
:1084F000400900200E00002005000020002A00088E
:10850000F80000201001002098010020000C01401C
:10851000B8000020D0000020BC000020DC000020BB
:1085200000140140C0000020022400222146641CE7
:108530006A540DE00020E5E500BF03240020A87088
:1085400006E0284602F056FD044601E00020D9E589
:1085500000BFF07820F018001030F070B6F801007D
:108560008108308861F3C9003080B6F8010020F43A
:10857000FE7000F58470A6F80100B07820F03E008F
:10858000801CB070601EC11700EB5171C910491CEE
:10859000728861F38A127280F07820F0E000F07047
:1085A00034810B21304600F0E1F838B90448006806
:1085B00040F48060024908600020A3E50120A1E5A5
:1085C0000000002001480078704700002A000020C9
:1085D00001480078704700002F000020704700001D
:1085E00070B504460D46214801F0F0FA002001F074
:1085F000B3FB012211021D4801F025FC00211B489C
:1086000001F0D8FA01221146184801F0B0FA05230A
:1086100022460021154801F0ADFB4FF460220121F4
:10862000124801F027FB01221146104801F003FB1C
:108630000E4801F0F7FA012001F0DAFE0B4801F0D4
:1086400081FA0121094801F0EFFB00BF0221074830
:1086500001F02CFB0128F9D1044801F0E1FB28804E
:108660000221024801F01EFB012070BD00240140E0
:108670002DE9F04705460E461548006800044FEA0C
:108680009018A8F5406000F10067002440F22539F9
:1086900002F08CF8FCF7A4FD384602F011F8FCF764
:1086A0009FFD01F0F7FF02F081F800BF0AE02819F2
:1086B000D0F800903819494602F09AF8FCF790FD7E
:1086C000201DC4B2B442F2DB01F0E4FFBDE8F08744
:1086D000E0F7FF1F10B50024FEF7C2FEC0B1FEF7A1
:1086E0001BFF98B10D4880680D498968884206D300
:1086F000FEF7CAFD08B102240EE001240CE0FEF7EB
:10870000C3FD08B1012407E0022405E0012403E0D1
:10871000FEF702FF00B10224204610BD38070020FA
:10872000B808002070B505460C461DB114B1B4F56B
:10873000807F01D9002070BD224629460748F9F7FD
:10874000FDFC0020064908800648046040F206311E
:10875000054803F0CAFA0120EDE70000B41000203C
:10876000E4000020E80000200044004070B586B01E
:1087700004460E4600252CB12648007810B926483C
:10878000007810B9002006B070BD2448216801604F
:108790002089224908810B461A8961685868F9F7CF
:1087A000CDFC142101A8F9F7E2FC1C480568E80893
:1087B000029004208DF80C0000208DF80D00174861
:1087C0000089082803DD08208DF80E0003E0134817
:1087D000007A8DF80E009DF80E20104841680DF1CA
:1087E0000F00F9F7ABFC01A90D4801F009FD0328C2
:1087F00001D10020C7E709484088C0F38410012850
:1088000006D00120034908700121054801F081FCD0
:108810000120B8E79C0000200D0000209A0E0020E7
:108820000064004070B505460C461DB114B1B4F5A6
:10883000807F01D9002070BD224629460948F9F7FA
:108840007DFC0020084908800848046040F2063199
:10885000074803F04AFA40F20631054803F052FA9D
:108860000120E8E7A40E0020A0000020A4000020C2
:108870000038014010B50448007800B110BD00F088
:1088800011F800BFFAE700002800002010B50448E6
:10889000007800B110BD00F0D9F800BFFAE7000081
:1088A0002D0000202DE9F041624C2546624F082042
:1088B00020706248007860704220A0701020E07044
:1088C0001620A0710020A080E07100212278501CA9
:1088D0002070A9542278501C2070A9542278501C72
:1088E0002070A9542278501C2070A9542278501C62
:1088F0002070A9542278501C2070A95497F8681051
:108900002278501C2070A95400212278501C20701D
:10891000A9542278501C2070A9542278501C207031
:10892000A9542278501C2070A9542278501C207021
:10893000A9542278501C2070A9542278501C207011
:10894000A9542278501C2070A95497F86800102868
:1089500054D2DFE800F008090A0B0C0D0E0F525339
:108960005310535317184AE049E048E047E046E007
:1089700045E044E043E06C20C15D2278501C20704B
:10898000A9543CE03BE02E4881782278501C2070AE
:10899000A9542B48408801122278501C2070A954F9
:1089A00000212278501C2070A9542278501C20707D
:1089B000A954234801792278501C2070A9542048DA
:1089C000808801122278501C2070A954002122783E
:1089D000501C2070A9542278501C2070A9541849AA
:1089E000CA882178481916490831F9F7A7FB207879
:1089F000134989790844207001E000E000BF00BFFE
:108A000022782146201DFCF753FC0646012E02D099
:108A10000020BDE8F08121782846FFF703FF012000
:108A2000084908700020488001200749087000BFED
:108A3000EFE700002C06002038070020220000206D
:108A4000100100202C070020280000202DE9F04113
:108A5000624C2546624F08202070624800786070A2
:108A60004220A0701020E0701620A0710020A0808D
:108A7000E07100212278501C2070A9542278501CEB
:108A80002070A9542278501C2070A9542278501CC0
:108A90002070A9542278501C2070A9542278501CB0
:108AA0002070A95497F868102278501C2070A9549F
:108AB00000212278501C2070A9542278501C20706C
:108AC000A9542278501C2070A9542278501C207080
:108AD000A9542278501C2070A9542278501C207070
:108AE000A9542278501C2070A9542278501C207060
:108AF000A95497F86800102854D2DFE800F008095C
:108B00000A0B0C0D0E0F52535310535317184AE013
:108B100049E048E047E046E045E044E043E06C20BF
:108B2000C15D2278501C2070A9543CE03BE02E48E7
:108B300081782278501C2070A9542B48408801125B
:108B40002278501C2070A95400212278501C2070DB
:108B5000A9542278501C2070A95423480179227806
:108B6000501C2070A9542048808801122278501C83
:108B70002070A95400212278501C2070A95422781A
:108B8000501C2070A9541849CA88217848191649E0
:108B90000831F9F7D3FA207813498979084420700D
:108BA00001E000E000BF00BF22782146201DFCF755
:108BB0009FFB0646012E02D00020BDE8F0812178FF
:108BC0002846FFF7AFFD01200849087000204880C3
:108BD00001200749087000BFEFE70000AC07002044
:108BE000B80800202C00002010010020AC08002054
:108BF0002D0000201048007820B10F484088401C0C
:108C00000D4948800D480078A0B10C484088401CB0
:108C10000A4948800846408841F28831884203DC8E
:108C200001200749087005E0044800210160002088
:108C30000349087070470000120000201600002051
:108C40001A0000200249097809B9024908717047E1
:108C5000E0000020A410002001200249087000203C
:108C6000488070477E0000200748007858B10648C9
:108C70004088401C80B204494880B0F5C87F02DBC0
:108C80000846002101607047D000002070B5024600
:108C900000231AE0002012E032F81060451C32F880
:108CA0001550AE4209DD32F81040451C32F815501F
:108CB00022F81050451C22F81540451CA8B2CD1AC8
:108CC0006D1E8542E8DC5D1CABB24D1E9D42E1DCB1
:108CD00070BD0000014800787047000029000020A6
:108CE00010B500F05FFC094800210160416081601F
:108CF00074210748F9F73BFA012006490870002063
:108D000048800520024981F8680010BD2C0700202A
:108D1000380700202400002007480078052809D2E1
:108D2000DFE800F003040506070003E002E001E0CD
:108D300000E000BF00BF7047290000200148007814
:108D4000704700002E00002010B500F081FC07489D
:108D5000002101604160816074210548F9F707FA3C
:108D60000520034981F8680010BD0000AC08002010
:108D7000B808002007480078052809D2DFE800F08D
:108D800003040506070003E002E001E000E000BF85
:108D900000BF70472E00002010B5B1480088401C6D
:108DA00080B2AF490880B0F57A7F1DDBAD4800681E
:108DB000401CAC4908600020A949088000BFAA48AF
:108DC000007878B1A8484088401C80B2A649488005
:108DD000012807DB00204880A448006840F02000FC
:108DE000A249086000BF00BFA148006820B1A048A8
:108DF0000068401E9E490860F9F74AFD00BF9D4883
:108E0000007890B19B48408828B19A484088401E1D
:108E10009849488009E09548006840F0010093496E
:108E20000860002093490870488000BF00BF924846
:108E3000007890B19048408828B18F484088401E03
:108E40008D49488009E08948006840F0040087495E
:108E50000860002088490870488000BFF9F7D4FCFA
:108E60008648007818B385484088401C80B2834902
:108E7000488096281BDB0020814908707F490870D4
:108E800048800846007918B90120087188600EE012
:108E90007A488068401C79498860032807D30020FD
:108EA00088607248006840F00800704908607548A2
:108EB000007818B373484088401C80B271494880DC
:108EC00096281BDB0020704908706E4908704880A6
:108ED0000846007918B90120087188600EE06948D9
:108EE0008068401C67498860032807D30020886099
:108EF0005E48006840F010005C49086063480078F4
:108F000020B362484088401C604948800846408839
:108F1000B0F5C87F0CDB002048805D48407802280F
:108F200014D05248006840F08000504908600DE0BD
:108F300056484088C82809D155484078012805D0AE
:108F40004A48006840F040004849086051480078AD
:108F500020B150484088401C4E4948804E484078D7
:108F600020B14D484088401C4B4948804B48007810
:108F700020B14A484088401C484948804848007809
:108F800020B147484088401C454948804548007802
:108F900020B144484088401C4249488042480078FB
:108FA00020B141484088401C3F4948803F480078F4
:108FB00020B13E484088401C3C4948803C480078ED
:108FC000D8B13B484088401C394948800846408811
:108FD000B0F5617F08DB01224021364801F0F4FC46
:108FE00000203349488008E031484088C82804DB25
:108FF000002240212F4801F0E7FC2F480078D8B12B
:109000002D484088401C2C49488008464088B0F5CF
:10901000617F08DB01228021264801F0D5FC002079
:109020002549488008E024484088C82804DB0022FD
:109030008021204801F0C8FCFAF754FCFAF788FCBC
:10904000FCF726F8F9F7D8FEFFF70EFEFBF742FC17
:10905000FFF7D0FDFCF7A8F8FCF766FB10BD000099
:109060008C0000208800002032000020000000203A
:1090700084000020A8000020EC0000202C07002025
:1090800028000020AC0800202D0000202400002033
:1090900010010020AC000020D8000020B00000200B
:1090A000B4000020B8000020BC000020C000002058
:1090B000C800002000100140CC00002010B514486A
:1090C000006840F0010012490860084640681149F4
:1090D00008400F494860084600680F4908400C499D
:1090E00008600846006820F4802008600846406850
:1090F0000A49084006494860084600680649084091
:10910000034908604FF41F00886002F065FA10BD43
:10911000001002400C00FFE8FFFFF6FEFFFF00F723
:1091200010B50121094802F0FDFC01280CD10121F4
:10913000064802F0F3FC4FF0804002F06DFC03485B
:1091400002F06AFCF9F73CFC10BD0000000400408E
:1091500010B511210148FFF709FB10BD20060020C2
:1091600010B504210148FFF701FB10BDC203002028
:1091700010B509210148FFF7F9FA10BDCC04002011
:1091800010B50D210148FFF7F1FA10BDD6050020FA
:1091900010B505211E4802F07CFD012818D11C489D
:1091A00002F020FDC4B21B480088FF2800D910BD82
:1091B00000210846FBF746FF164801880088401C3E
:1091C000144A10801448445405210120FBF73AFF4B
:1091D00006210F4802F05DFD012816D10F480088D6
:1091E0000F490968884205D340F20631084802F069
:1091F0006FFDDCE7094802880088401C074B188097
:109200000848815C024802F0F2FC00BFCFE7000092
:1092100000380140A2000020A40F0020A000002080
:10922000A4000020A40E002010B505211E4802F065
:1092300030FD012818D11C4802F0D4FCC4B21B48F0
:109240000088FF2800D910BD00210846FBF708FF61
:10925000164801880088401C144A10801448445461
:1092600005210120FBF7FCFE06210F4802F011FD4D
:10927000012816D10F4800880F490968884205D394
:1092800040F20631084802F023FDDCE70948028875
:109290000088401C074B18800848815C024802F097
:1092A000A6FC00BFCFE7000000440040E60000201D
:1092B000B4110020E4000020E8000020B4100020D9
:1092C00010B586B000242D488078C0F344002B49A7
:1092D0004988C1F38411884246D0284880784008E4
:1092E000401C2649897860F3450124488170142187
:1092F00001A8F8F73CFF21480468E0080290042028
:109300008DF80C0000208DF80D001C488078C0F30B
:10931000440020B119488078C0F3440000E02020C8
:10932000441EE40015488078C0F34400134949887E
:10933000C1F38411884203D008208DF80E0005E0A7
:109340000E48007A001BC0B28DF80E009DF80E206A
:109350000A48406801190DF10F00F8F7EFFE01A966
:10936000074800F04DFF06E0002006490870012183
:10937000034800F0CAFE06B010BD00009A0E00209F
:10938000006400409C00002070B586B001AA002156
:10939000394800F0C2FE9DF8170020B1012806D020
:1093A00002280CD107E0354C4FF4807609E0344CAC
:1093B0004FF4807605E0334C4FF4807601E006B040
:1093C00070BD00BF9DF80C00029940EAC1009DF8F5
:1093D0000D1040EA01052560A078C0F3440018B1E3
:1093E000A078C0F3440000E020206188C1F384111C
:1093F00019B16188C1F3841100E02021884200DDA9
:10940000DDE76088C0F3841018B16088C0F3841071
:1094100000E02020C500B54200D9D0E7A078C0F315
:10942000440018B1A078C0F3440000E02020451E9D
:10943000616801EBC5009DF80E200DF10F01F8F7F2
:109440007DFEA078C0F3440018B1A078C0F34400BA
:1094500000E020206188C1F3841119B16188C1F353
:10946000841100E02021884204D19DF80E0000EB19
:10947000C500208100BFA2E7006400407C0E0020F0
:10948000860E0020900E00202DE9F041054640F2A6
:10949000DC5725B1012D05D0022D0DD107E00020AC
:1094A000BDE8F0810E20194981F8680006E00F2020
:1094B000164981F8680001E00020F1E700BF144878
:1094C000006820F0010012490860FFF7EBF9002660
:1094D000002413E00A2000F08BFF0D48007800F014
:1094E000010048B10A48006820F0010008490860FE
:1094F000FDF7C8FCC6B206E0601C84B20A2097FBE8
:10950000F0F0A042E6DC00BF70B2C9E738070020E7
:10951000000000202DE9F041054640F2DC5725B15E
:10952000012D05D0022D0DD107E00020BDE8F0810E
:109530000E20194981F8680006E00F20164981F8CD
:10954000680001E00020F1E700BF1448006820F047
:10955000040012490860FFF779FA0026002413E09E
:109560000A2000F045FF0D48007800F0040048B1E3
:109570000A48006820F0040008490860FDF7D8FC9C
:10958000C6B206E0601C84B20A2097FBF0F0A0424D
:10959000E6DC00BF70B2C9E7B80800200000002078
:1095A00000BFFEE710B540F2026001F009FF4FF482
:1095B000C06001F005FF40F20E6001F001FF4FF4C2
:1095C000007303221821204801F050FA4FF4806301
:1095D000032204211C4801F049FA1C4802F00CFB4C
:1095E0004FF41641194802F0B5FA0021174802F06D
:1095F000C5FB0021154802F0B1FB0021134802F021
:109600009DFB0021114802F05BFB00210F4802F096
:109610004FFB04210D4802F099FB08210B4802F092
:10962000A5FB4FF4407001F0A9FC00220121252088
:1096300001F04EFC40F20531044802F056FB0348AD
:1096400002F022FB10BD000000080140003801407C
:1096500010B540F2026001F0B3FE4FF4C06001F0BB
:10966000AFFE042303221821214801F0FFF908234B
:10967000032204211E4801F0F9F940F2117001F0B3
:109680009FFE1C4802F0B8FA4FF41641194802F048
:1096900061FA0021174802F071FB0021154802F021
:1096A0005DFB0021134802F049FB0021114802F044
:1096B00007FB00210F4802F0FBFA04210D4802F0DD
:1096C00045FB08210B4802F051FB4FF4407001F0BC
:1096D00055FC00220121262001F0FAFB40F2053161
:1096E000044802F002FB034802F0CEFA10BD00006D
:1096F00000080140004400402DE9F04105461348B0
:10970000006800048609A6F5805000F100673DB1AD
:1097100042F2233401200E4908700020488001E005
:109720004FF6FF7401F042F8FBF7ACFE384600F04C
:10973000C7FFFBF7A7FE2146384600F04BFFFBF7BB
:10974000A1FE00F0A7FFBDE8F0810000E0F7FF1FD9
:109750007A0000202DE9F04105461A48006800040F
:109760004FEA9018A8F5006000F1006600244FF65B
:10977000FF7701F01BF8FBF733FD304600F0A0FF48
:1097800000BF0FE0FBF72CFD601C2F5C4FF6FF7055
:1097900000EA0727285D07433019394600F01AFF11
:1097A000A01CC4B2122CEDDB00F074FFA8F5006021
:1097B00000F10066122231460348F8F7BFFCBDE80D
:1097C000F0810000E0F7FF1FF800002010B540F224
:1097D000036001F0F5FD4FF46043032210210248BD
:1097E00001F044F910BD0000000C014010B540F23A
:1097F000046001F0E5FD0823032210210A4801F06E
:1098000035F940F2026001F0DBFD40F2096001F041
:10981000D7FD032001F078FC03231A4600210348FA
:1098200001F024F910BD00000010014000080140C3
:1098300010B5202303220021014801F017F910BDC3
:10984000000801400FB4054B10B503A9044A029863
:1098500000F018F810BC5DF814FB0000B1A8000877
:10986000F400002002E008C8121F08C1002AFAD143
:1098700070477047002001E001C1121F002AFBD190
:10988000704700002DE9FF4F8DB09B460F46044600
:10989000002606E025280BD05A460F999047641CF5
:1098A000761C20780028F5D111B03046BDE8F08F45
:1098B0000025A8460122984900E0054314F8013F1D
:1098C000203B02FA03F00842F7D120782E2817D166
:1098D00014F8010F45F004052A280ED06FF02F026E
:1098E0002078A0F1300109290AD808EB880102EBA1
:1098F000410100EB0108641CF2E757F8048B641C7B
:1099000020786C280DD004DC4C2812D06A2811D1A4
:1099100004E074280DD07A280CD10AE045F4001533
:1099200007E0617845F48015814202D1641C05F599
:109930008015641C2278692A45D008DC002AB3D03F
:10994000582A69D0632A10D0642A08D13BE0702AD3
:1099500067D0732A13D0752A5CD0782A5CD0104661
:109960005A460F999047761CD3E017F8040B8DF8F0
:10997000000000208DF80100E946012003E057F8BF
:10998000049B4FF0FF3069074FF0000501D40AE057
:109990006D1C45450DDA8542FADB19F805100029E2
:1099A000F6D106E06D1C8542FCDB19F80510002994
:1099B000F8D12E4404E019F8010B5A460F9990474C
:1099C0006D1EF8D2A5E00A200021CDE90801C5F3FB
:1099D000025002280DD001CFC117031E71F1000300
:1099E0000DDA4FF0000CD0EB0C006CEB01012D23D5
:1099F00008E0FF1D27F00707F7E80201EDE72B0558
:109A000004D52B238DF8283001233BE0EB0739D018
:109A10002023F7E70A2000E010200021CDE908010B
:109A200007E01020002145F00405CDE908014FF0C2
:109A30000808C5F3025002280FD001CF00214FF0D3
:109A4000000A2B071FD5702A0DD0DDE908C38CF062
:109A5000100C5CEA030C0CD015E0FF1D27F0070783
:109A6000F7E80201EBE740228DF828204FF0010AC9
:109A70000BE050EA010306D030238DF828308DF832
:109A8000292002239A46582A04D024A20DF1200945
:109A90000B9209E026A2F9E7DDE90823F8F788FD33
:109AA0000B9B9B5C09F8013D50EA0102F4D1ADEB40
:109AB000090020300890680701D44FF00108089988
:109AC000884502DDA8EB010000E00020804600256B
:109AD00006E00AA85A46405D0F9990476D1C761C17
:109AE0005545F6DB04E030205A460F999047761C26
:109AF000B8F10001A8F10108F5DC05E019F8010B47
:109B00005A460F999047761C0899481E08900029DC
:109B1000F4DC641CC5E60000092801003031323352
:109B20003435363738396162636465660000000099
:109B30003031323334353637383941424344454683
:109B400000000000816841F00801816000BF816869
:109B500001F008010029FAD1816841F00401816017
:109B600000BF816801F004010029FAD1704730B5C7
:109B7000012902D002291AD10CE0C36A23F4700330
:109B8000C362C36A541E4FF4700505EA04542343AC
:109B9000C3620DE0836B23F440138363836B541E15
:109BA0004FF4401505EA04542343836300E000BFEB
:109BB00000BF30BD21B1826842F40062826003E0E0
:109BC000826822F4006282607047000010B504468B
:109BD0001348204430B1B0F5806F0CD0B0F5C05FB1
:109BE0001BD111E040F2093001F00AFC40F20930CB
:109BF00001F0F6FB12E040F20A3001F001FC40F205
:109C00000A3001F0EDFB09E040F20F3001F0F8FB03
:109C100040F20F3001F0E4FB00E000BF00BF10BDD8
:109C200000DCFEBF816801F0010119B9816841F0D3
:109C300001018160704772B101F001031BB18368BB
:109C400043F48013836001F0020393B1836843F40B
:109C5000004383600DE001F001031BB1836823F42E
:109C60008013836001F002031BB1836823F4004377
:109C700083607047012902D0022910D107E0836870
:109C800023F46023836083681343836008E0836860
:109C900023F4E043836083681343836000E000BFE4
:109CA00000BF704702688A43026070470246002086
:109CB00013680B4003B1012070472DE9FE4F824627
:109CC0000D461DB96FF00100BDE8FE8F00240EE0C7
:109CD000684600EB44015046FEF782FC8146B9F12C
:109CE000000F02DC6FF00200EEE7601CC4B2062C2D
:109CF000EED30026002701240FE03DF816003DF8C2
:109D00001410884200DD26463DF817003DF8141077
:109D1000884200DA2746601CC4B2062CEDD3BE424E
:109D200004D1BDF8000028800120CDE74FF00008E5
:109D300000240BE0B44207D0BC4205D03DF814002B
:109D400008EBA0001FFA80F8601CC4B2062CF1D307
:109D5000A5F800800120B7E70549096821F47021C2
:109D6000034A116011460968014311607047000001
:109D700004240140F0B51D4606290CDA436B01EBC3
:109D800081071F26BE40B34301EB810602FA06F6A7
:109D90003343436322E00C290EDA036B8E1F06EB7C
:109DA00086071F26BE40B3438E1F06EB860602FAC7
:109DB00006F63343036311E010290FDAC36AA1F1F9
:109DC0000C0606EB86071F26BE40B343A1F10C0626
:109DD00006EB860602FA06F63343C3620A2A0CDA59
:109DE000046902EB42070726BE40B44302EB420679
:109DF00005FA06F63443046111E0122A0FDAC4684A
:109E0000A2F10A0606EB46070726BE40B443A2F1BC
:109E10000A0606EB460605FA06F63443C460F0BDB2
:109E20000146C86C80B2704701F001021AB1826825
:109E300042F48002826001F002021AB1826842F4A8
:109E4000001282607047AAB101F480731BB14368AD
:109E500043F48073436001F480631BB1436843F4AF
:109E60008063436001F00203CBB1836843F00203D7
:109E7000836014E001F480731BB1436823F48073A2
:109E8000436001F480631BB1436823F48063436043
:109E900001F002031BB1836823F002038360704763
:109EA00010B501F05FF901F053F910BD10B504468B
:109EB0000548844207D140F2194001F0A1FA40F26E
:109EC000194001F08DFA10BD0064004001460020E9
:109ED0008A69C2F30210704710B50021837A01220B
:109EE00002FA03F13E4A126842F001023C4B1A604A
:109EF0003B4A1C3212688A43394B1C331A60C289B0
:109F0000DAB9374A0C3212688A43354B0C331A607F
:109F1000C288344B03EA024243881A434389304CD7
:109F2000403444F8332082882E4B03EA02420388EF
:109F30001A43438904EBC3035A60C289012A1BD127
:109F4000274A0C3212680A43254B0C331A600288E8
:109F5000244B03EA024243881A434389204C40348D
:109F600044F8332082881F4B03EA0242C3881A4315
:109F7000438904EBC3035A6082893AB9184A121D17
:109F800012688A43164B1B1D1A6006E0144A121D04
:109F900012680A43124B1B1D1A6002893AB9104A13
:109FA000143212688A430E4B14331A6006E00C4ACE
:109FB000143212680A430A4B14331A60027C012AD5
:109FC00006D1074A1C3212680A43054B1C331A603B
:109FD000034A126822F00102014B1A6010BD000012
:109FE000006600400000FFFF70B502464FF6FF73A9
:109FF0000020146824F002041460146844F0010482
:10A00000146000E05B1E546804F001040CB9002BDE
:10A01000F8D1546804F001040CB9002074E00C7805
:10A020004FF0404505EA84744D784FF0407606EADB
:10A0300005652C438D784FF4702606EA05452C43C0
:10A04000CD784FF4E00606EA05552C434D896D1E88
:10A05000C5F309052C43D4610C79012C04D1146893
:10A0600044F08004146003E0146824F08004146059
:10A070004C79012C04D1146844F04004146003E0CE
:10A08000146824F0400414608C79012C04D1146805
:10A0900044F02004146003E0146824F020041460E9
:10A0A000CC79012C04D1146844F01004146003E04E
:10A0B000146824F0100414600C7A012C04D1146884
:10A0C00044F00804146003E0146824F008041460E9
:10A0D0004C7A012C04D1146844F00404146003E0A9
:10A0E000146824F004041460146824F0010414605B
:10A0F0004FF6FF7300E05B1E546804F001040CB1DE
:10A10000002BF8D103B1012070BD42698A4342613E
:10A11000704742690A434261704710B500F5D87331
:10A1200003EB01131B6803F004031372137A3BB9AA
:10A1300000F5D87303EB01131B685B0D136006E099
:10A1400000F5D87303EB01131B68DB08536000F5BF
:10A15000D87303EB01131B6803F00203537200F57D
:10A16000DA7303EB01131B681B0AD37400F5DA736F
:10A1700003EB01131B6803F00F03937200F5DC730C
:10A1800003EB01131B68D37200F5DC7303EB0113BF
:10A190001B681C0A147300F5DC7303EB01131B68C6
:10A1A0001C0C547300F5DC7303EB01131B681C0ECD
:10A1B000947300F5DE7303EB01131B68D37300F592
:10A1C000DE7303EB01131B681C0A147400F5DE73C5
:10A1D00003EB01131B681C0C547400F5DE7303EBD6
:10A1E00001131B681C0E947421B9C36843F020034B
:10A1F000C36003E0036943F02003036110BD000066
:10A2000030B502460B460021906800F08060B0F146
:10A21000806F00D110E0906800F00060B0F1006F36
:10A2200001D1012108E0906800F08050B0F1805F1A
:10A2300001D1022100E00321032901D1032030BD17
:10A2400002F5C07000EB0110006800F0010402F597
:10A25000C07000EB01100460187A88B918883B4C74
:10A2600004EA40505C7A204302F5C07404EB011408
:10A270002468204302F5C07404EB0114206013E04D
:10A280006FF00704586804EAC0001C7A20435C7A27
:10A29000204302F5C07404EB01142468204302F546
:10A2A000C07404EB0114206002F5C27000EB0110D1
:10A2B000006820F00F0402F5C27000EB011004608A
:10A2C00002F5C27000EB011000689C7A204302F591
:10A2D000C27404EB01142060987B4FF07F4404EAC1
:10A2E00000605C7B4FF47F0505EA044420431C7B3F
:10A2F0002D1205EA04242043DC7A204302F5C474BD
:10A3000004EB01142060987C2C0404EA00605C7C5F
:10A310002D0205EA044420431C7C2D1205EA042486
:10A320002043DC7B204302F5C67404EB011420605B
:10A3300002F5C07000EB0110006840F0010402F566
:10A34000C07000EB01100460084678E70000E0FFF1
:10A3500010B5024632B1012A16D0022A20D0032AB3
:10A3600041D12EE000234B71CB718B7140F2FF3352
:10A370004B8100230B724B7002238B700023CB7038
:10A380000B714B720B7030E00123CB8100230B74F7
:10A390000B810B804B808B80CB808B814B8124E0A9
:10A3A000002005E0002401F10B031C54431CD8B22B
:10A3B0000828F7D300238B724B600B724B720B6033
:10A3C00013E0002005E0002401F10B031C54431CA2
:10A3D000D8B20828F7D300238B724B600B72CB7472
:10A3E0004B720B6001E000BFFEE700BF10BD000034
:10A3F0000349086000BF024909680029FBD1704782
:10A400008400002000EB400100BF0A1EA1F1010101
:10A41000FBD1704710B52C4B1B6883432A4C23603B
:10A42000231D1B688343241D2360231D1B68834356
:10A43000241D2360231D1B688343241D236011B149
:10A4400001290ED105E0204B1B6803431E4C2360FD
:10A4500008E01D4B1B1D1B6803431B4C241D236080
:10A4600000E000BF00BF22B1012A0FD0022A27D18D
:10A4700019E0154B08331B680343134C0834236061
:10A48000231D1B688343241D23601AE00E4B0833F1
:10A490001B6883430C4C08342360231D1B68034353
:10A4A000241D23600DE0084B08331B680343064C52
:10A4B00008342360231D1B680343241D236000E030
:10A4C00000BF00BF10BD0000000401400249096840
:10A4D0000143014A116070470004014001490860CE
:10A4E000704700001404014001460748006800EA74
:10A4F000010205481438006800EA010312B10BB1EB
:10A50000012070470020FCE71404014000B5034619
:10A51000012200BF00F00CF802465B1E012A01D1A7
:10A52000002BF7D1012A00D10422104600BD000003
:10A5300000200A49C96801F0010109B101200CE0BD
:10A540000649C96801F0100109B1032005E003497B
:10A55000C96801F0040101B10220704700200240E7
:10A5600000B50346012200BF00F00CF802465B1E56
:10A57000012A01D1002BF7D1012A00D10422104673
:10A5800000BD000000200A49C96C01F0010109B1B9
:10A5900001200CE00649C96C01F0100109B103204B
:10A5A00005E00349C96C01F0040101B102207047C4
:10A5B00000200240064A02EB9011096800F01F03D8
:10A5C00001229A401143024B03EB90121160704735
:10A5D0000020024070B504460D4600262A48008837
:10A5E000B0F5007F35D22948844219D24FF470204B
:10A5F000FFF78CFF0646002E43D12548006940F046
:10A6000001002349086125804FF47020FFF77EFF89
:10A6100006461F48006920F001001D49086130E02E
:10A620004FF47020FFF79CFF064656BB1848006D9C
:10A6300040F001001649086525804FF47020FFF7AF
:10A640008FFF06461248006D20F001001049086592
:10A6500017E04FF47020FFF759FF06468EB90C48FB
:10A66000006940F001000A49086125804FF470201C
:10A67000FFF74CFF06460648006920F00100044938
:10A680000861304670BD0000E0F7FF1FFFFF0708BC
:10A69000002002400848006940F080000649086137
:10A6A00006480088B0F5007F04D90846006D40F0E8
:10A6B000800008657047000000200240E0F7FF1F9F
:10A6C00030B5054636480088B0F5007F48D9354892
:10A6D00085421ED24FF47020FFF718FF0446002C6D
:10A6E0005BD13148006940F002002F4908610846FB
:10A6F0004561006940F0400008614FF47020FFF7A9
:10A7000005FF04462848006920F002002649086138
:10A7100043E04FF47020FFF723FF0446002C3CD1A8
:10A720002148006D40F002001F4908650846456554
:10A73000C06900F0020008B1084645611A48006D82
:10A7400040F04000184908654FF47020FFF708FFFB
:10A7500004461548006D20F00200134908651CE00E
:10A760004FF47020FFF7D2FE0446B4B90E480069DA
:10A7700040F002000C49086108464561006940F05C
:10A78000400008614FF47020FFF7C0FE0446064801
:10A79000006920F0020004490861204630BD000035
:10A7A000E0F7FF1FFFFF0708002002400C48006988
:10A7B00000F0800020B10B48094948600A48486011
:10A7C0000A480088B0F5007F09D90548006D00F0FF
:10A7D000800020B103480249486403484864704738
:10A7E0000020024023016745AB89EFCDE0F7FF1F52
:10A7F00070B504460D4600262A480088B0F5007F53
:10A8000035D92948844219D24FF47020FFF77EFED3
:10A810000646002E43D12548006940F00100234937
:10A82000086125604FF47020FFF770FE06461F4850
:10A83000006920F001001D49086130E04FF47020EC
:10A84000FFF78EFE064656BB1848006D40F001002B
:10A850001649086525604FF47020FFF781FE064613
:10A860001248006D20F001001049086517E04FF410
:10A870007020FFF74BFE06468EB90C48006940F089
:10A8800001000A49086125604FF47020FFF73EFE81
:10A8900006460648006920F0010004490861304678
:10A8A00070BD0000E0F7FF1FFFFF07080020024017
:10A8B00030B585B004460D4610480078D8B1142153
:10A8C0006846F7F754FC42F24510019004208DF8D9
:10A8D000080000208DF8090001208DF80A00E0B280
:10A8E0008DF80B0069460648FFF78AFC4FF4FA70B2
:10A8F000FFF788FD00BF204605B030BD0D000020E9
:10A900000064004038B50020009000250122082195
:10A91000284800F059F82848007800F0010026493E
:10A9200008700846007810B1012804D101E0002524
:10A9300006E0012504E000201F490870002500BF43
:10A9400000BF69462846FFF7B8F9012800D025E086
:10A9500000220821174800F037F8BDF800004FF634
:10A96000FF7101EA001000907D2414E0134830F8D4
:10A970001400BDF8001088420BDBA4F1280041B29E
:10A980000D4802780078401C0B4B18700C4881541D
:10A9900038BD601E84B2002CE8D100BF00210648FB
:10A9A00002780078401C044B18700548815400BFA1
:10A9B000EEE7000000100140380000208CBD0008C8
:10A9C00036000020416170470AB1016100E0416139
:10A9D0007047000010B500228B071C0F0F2303FAED
:10A9E00004F204290EDA204B9B6893431E4CA360AB
:10A9F00023469B688C07240F00FA04F423431A4C67
:10AA0000A3602FE008290EDA174BDB689343164C3E
:10AA1000E3602346DB688C07240F00FA04F4234329
:10AA2000114CE3601EE00C290EDA0F4B1B699343B7
:10AA30000D4C236123461B698C07240F00FA04F494
:10AA40002343094C23610DE0074B5B699343064C9C
:10AA5000636123465B698C07240F00FA04F42343E7
:10AA6000014C636110BD000000000140F0B50446D8
:10AA700016460025002201F00F0501F0100707B16E
:10AA8000354300201EE0012787401F40C7B12268E0
:10AA90004FEA800C0F2707FA0CF7BA43870005FA34
:10AAA00007F73A43282904D1012787401F406761EF
:10AAB00005E0482903D1012787401F402761226014
:10AAC000471CB8B20828DED3082022E001278740BF
:10AAD0001F40E7B16268A0F108074FEA870C0F2713
:10AAE00007FA0CF7BA43A0F10807BF0005FA07F709
:10AAF0003A43282904D1012787401F40676105E0B8
:10AB0000482903D1012787401F4027616260471C05
:10AB1000B8B21028DAD3F0BD02469068084008B1F8
:10AB2000012070470020FCE70246D068084008B1C9
:10AB3000012070470020FCE7F0B50A4600230024FE
:10AB40000021002500F00046B6F1004F02D11D4E55
:10AB5000F16901E01B4E7168C0F3034583B200F454
:10AB60004016B6F5401F08D121F07061154E766889
:10AB700026F07066134F7E6012E000F48016B6F582
:10AB8000801F06D1032606FA05F4A14341F0706147
:10AB900006E0460D360103FA06F6B14341F0706156
:10ABA00022B1460D360103FA06F6314300F00046A5
:10ABB000B6F1004F02D1034EF16101E0014E716028
:10ABC000F0BD00000000014000F018FDFCF755FD4D
:10ABD000FEF786F8FEF7B8F8F9F748FAFCF716FD25
:10ABE000FCF745FDF9F74CF8FAF748FAF7F700FEDD
:10ABF000FAF720FDF7F7E6FFF9F794FFFCF702FDFF
:10AC0000AF4800F047FA00BFF9F778FDF9F734FDD7
:10AC1000FCF76EFBF9F7A8FDFEF77EF8FEF7AAF841
:10AC2000F9F7BCFFF9F7E6FFF9F760FEF9F78AFDDF
:10AC3000F9F732F8A348007800F0400038B1FDF78A
:10AC400019FEA048006820F040009E4908609D4819
:10AC5000007800F0800038B1FDF718FE99480068D0
:10AC600020F08000974908609648008800F48070C2
:10AC700040B1FCF7E1FE28B19248006820F48070F2
:10AC8000904908608F48008800F4007040B1FCF7DC
:10AC9000DBFE28B18B48006820F400708949086009
:10ACA0008848008800F4806040B1FCF7D5FE28B1E8
:10ACB0008448006820F480608249086081480088E8
:10ACC00000F4006040B1FCF7AFFE28B17D48006899
:10ACD00020F400607B490860FBF76CFB7948007842
:10ACE00000F0200038B1FFF70DFE7648006820F034
:10ACF0002000744908607348007800F0080038B1FB
:10AD0000FCF7C4FD6F48006820F008006D4908603A
:10AD10006C48007800F0100038B1FCF7EDFD694890
:10AD2000006820F01000674908606648007800F06D
:10AD3000010038B1FCF7A6F86248006820F0010075
:10AD4000604908605F48007800F0040038B1FCF703
:10AD5000EFF85C48006820F004005A490860594840
:10AD6000008800F4805038B1FEF7FAF955480068C1
:10AD700020F48050534908605248008800F4005085
:10AD800038B1FEF7F5F94F48006820F400504D49FE
:10AD900008604C48008800F4804038B1FEF7F0F9B4
:10ADA0004848006820F480404649086045480088CB
:10ADB00000F4004038B1FEF7CBF94248006820F4B7
:10ADC0000040404908603F48006800F4803038B1D6
:10ADD000F7F7D6FD3B48006820F480303949086019
:10ADE0003848006800F4003038B1F7F799FE35486C
:10ADF000006820F40030334908603248006800F4ED
:10AE0000802048B1F7F7A0FDF7F7D4FE2D48006881
:10AE100020F480202B4908602A48006800F40020B4
:10AE200038B1F7F79FFD2748006820F40020254936
:10AE300008602448006800F4001038B1FAF75EF9A1
:10AE40002048006820F400101E4908601D48006872
:10AE500000F4801028B11B48006820F480101949C4
:10AE600008601848006800F4800000283FF4CCAE69
:10AE70001448006820F4800012490860012080F323
:10AE8000138800BF00BF00BF00BF00BF00BFBFF3FB
:10AE90004F8F00BF00BF00BF0B48006800F4E060A8
:10AEA0000A490843001D0849086000BF00BF00BFF1
:10AEB000BFF34F8F00BF00BF00BF00BFFEE7000021
:10AEC00044332211000000200CED00E00000FA05E0
:10AED0002DE9F04103460D46164600240027A04602
:10AEE0002448006800F4E060B0F5A06F15D006DCDF
:10AEF000B0F5407F18D0B0F5806F19D110E0B0F5F3
:10AF0000C06F06D0B0F5E06F12D100274FF00408F3
:10AF100015E001274FF0030811E00227B8460EE0C4
:10AF200003274FF001080AE004274FF0000806E06D
:10AF30004FF4A06000F022F80227B84600BF00BF1F
:10AF4000C7F1040005FA00F4C8F104010F20C8405D
:10AF50003040044324010848C45403F01F01012079
:10AF600088405911890001F1E021C1F80001BDE8D4
:10AF7000F08100000CED00E000E400E00249014334
:10AF8000024A1160704700000000FA050CED00E075
:10AF90000348006840F48070014908607047000071
:10AFA000007000400E4A126822F003020C4B1A6037
:10AFB0001A46126802431A600A4A126842F00402F2
:10AFC000084B1A6009B930BF02E040BF20BF20BF64
:10AFD000044A126822F00402024B1A607047000013
:10AFE0000070004010ED00E010B540F20730FFF7B0
:10AFF000E1FA10BD2DE9F041044620790004E17822
:10B0000040EA0120A17840EA010707F100663046D6
:10B01000F7F7B8F80546FA2D00DDFA2520796071BA
:10B02000E0782071A078E0700020A0702A463146B8
:10B03000A01DF7F783F8A81DC0B2BDE8F08100009D
:10B040004FF0FF3000F026F8012080F3138800BF96
:10B0500000BF00BF00BF00BF00BFBFF34F8F00BFE6
:10B0600000BF00BF0948006800F4E06008490843D9
:10B07000001D0649086000BF00BF00BFBFF34F8F2F
:10B0800000BF00BF00BF00BFFEE700000CED00E006
:10B090000000FA052DE9F04705461A48006800044B
:10B0A0004FEA9019A9F5806000F10064D4F8088097
:10B0B000454501D1BDE8F08726686768FFF776FB54
:10B0C00008F1010080B1FFF78FFF2046FFF7F8FA83
:10B0D000FFF78AFF31462046FFF78AFBFFF784FF20
:10B0E0003946201DFFF784FB681C30B1FFF77CFF59
:10B0F000294604F10800FFF77BFBFFF7CBFA00BFFE
:10B10000D8E70000E0F7FF1F0F4A51680F4A1140CF
:10B11000082814D2DFE800F004050607130A130B11
:10B1200000BF00BF00BF41EA803109E000BF20F04E
:10B1300004004FF0805242EA8032114300E000BF29
:10B1400000BF014A5160704700100240FF3FFFEF0F
:10B150000348006A20F4803001490862704700000B
:10B16000001002400348006A40F480300149086240
:10B1700070470000001002402DE9F04F8BB00746E9
:10B18000002009903EA090E8004CC068CDE905BEC3
:10B19000CDF810A007900FF2EC0ADAE9000ACDE929
:10B1A000020A0FF2E00ADAE9000ACDE9000A38489B
:10B1B0004068C0F381000A900A9820B1012804D0A9
:10B1C000022829D103E0334928E0324926E03048FB
:10B1D000406800F48038B8F5803F09D12D4C2C48E8
:10B1E000406800F40039B9F5003F02D1641000E076
:10B1F000294C27484068C0F383422548406800F046
:10B20000006008B142F010020F2A01D2921C00E047
:10B21000521C04FB02F101E01E4900BF00BF1C48A4
:10B220004068C0F3031504A8465D21FA06F31848E8
:10B230004068C0F3022502A8465D23FA06FC1448C4
:10B240004068C0F3C2251DF8056023FA06F0089097
:10B2500037B1012F06D0022F06D0032F0AD106E006
:10B26000099108E0099306E0CDF824C003E00898AE
:10B27000099000E000BF00BF09980BB0BDE8F08F57
:10B280000000000000000000010203040607080996
:10B290000010024000127A0000093D000146074AF2
:10B2A00002EB9110006801F01F0301229A40104048
:10B2B00008B1012070470020FCE7000000100240A8
:10B2C000064A02EB9011096800F01F0301229A4020
:10B2D0001143024B03EB90121160704700100240C3
:10B2E000F0B50646002400270025182E51D003DCB7
:10B2F0006EB3102E5DD106E0B6F5006F14D0B6F532
:10B30000106F56D133E004E01120FFF7C7FF054668
:10B31000641C1DB94FF6FF708442F5D11120FFF770
:10B32000BDFF00B1012745E005E040F60100FFF751
:10B33000B5FF0546641C1DB96FF07C408442F4D112
:10B3400040F60100FFF7AAFF00B1012732E004E058
:10B350000120FFF7A3FF0546641C15B9B4F5A06FE3
:10B36000F6D10120FFF79AFF00B1012722E005E0A6
:10B3700040F60110FFF792FF0546641C15B90F480F
:10B380008442F5D140F60110FFF788FF00B1012794
:10B3900010E004E01920FFF781FF0546641C15B991
:10B3A00006488442F6D11920FFF778FF00B1012743
:10B3B00000E000BF00BF3846F0BD0000FFFF0F00F7
:10B3C000064A02EB9011096800F01F0301229A401F
:10B3D0001143024B03EB90121160704700100240C2
:10B3E000064A02EB9011096800F01F0301229A40FF
:10B3F0009143024B03EB9012116070470010024022
:10B40000064A02EB9011096800F01F0301229A40DE
:10B410001143024B03EB9012116070470010024081
:10B42000044A116A21F4407141EA0002014B1A6298
:10B43000704700000010024000B5024600F00CF812
:10B44000100C0449086090B2091D086000F00EF865
:10B4500000BD0000202800400348006840F01000B4
:10B460000149086070470000042800400348006854
:10B4700020F01000014908607047000004280040D7
:10B4800000B50246FFF7E8FF100C0449086090B2CF
:10B49000091D0860FFF7EAFF00BD00001828004002
:10B4A000024909688143014A11607047042800403D
:10B4B000014604480068084008B101207047002098
:10B4C000FCE7000004280040024909680143014AE2
:10B4D000116070470028004000BF0348006800F07A
:10B4E00020000028F9D070470428004000B502462B
:10B4F000FFF7B2FFC2F303400349086090B2091D91
:10B500000860FFF7B3FF00BD082800400648006848
:10B5100020F008000449086000BF0348006800F0FC
:10B5200008000028F9D070470428004000200021BE
:10B53000264A126842F00102244B1A6000BF401CE8
:10B54000224A126802F0020111B9B0F5A06FF6D1DB
:10B550001E4A126802F002020AB900BFFEE71B4A47
:10B5600052681A4B5A601A4652685A601A46526814
:10B5700042F480625A601A465268154B1A40134BC7
:10B580005A601A465268134B1A43104B5A601A46B7
:10B59000126842F080721A6000BF0C4A126802F012
:10B5A0000072002AF9D0094A526822F00302074BC0
:10B5B0005A601A46526842F002025A6000BF034ABB
:10B5C000526802F00802002AF9D0704700100240C9
:10B5D000FFFFC3F70000280810B5FFF7A7FF10BD55
:10B5E0004FF0E020006920F002004FF0E0210861F8
:10B5F0000846006920F001000861704710B5144842
:10B6000000684FF47A71B0FBF1F4601EB0F1807FF6
:10B6100001D301200FE0601E4FF0E02148610F21AF
:10B620004FF0FF30FCF72EF800204FF0E02188614A
:10B6300007200861002008B100BFFEE70021481E76
:10B64000FCF720F80020034908600349088010BD7A
:10B65000F0000020840000208C000020016841F0F0
:10B66000800101607047000010B531B101293FD061
:10B6700002297DD003297CD1BFE0036A23F00103B6
:10B680000362836923F003038361036A14882343FD
:10B690000362036A23F002030362036A948823436C
:10B6A00003626A4B984202D0694B98421FD1036AE9
:10B6B00023F004030362036A548823430362036A8A
:10B6C00023F008030362036AD488234303624368B8
:10B6D00023F48073436043681489234343604368C1
:10B6E00023F4007343604368548923434360ABE011
:10B6F000036A23F010030362836923F440738361B8
:10B70000036A148843EA04130362036A23F02003E4
:10B710000362036A948843EA041303624B4B984222
:10B7200002D04B4B984226D1036A23F040030362B8
:10B73000036A548843EA04130362036A23F0800314
:10B740000362036AD48843EA04130362436823F460
:10B75000806343604368148943EA84034360436819
:10B7600023F4006343604368548943EA840301E09F
:10B7700002E068E0436067E0036A23F480730362D9
:10B78000C36923F00303C361036A148843EA0423F3
:10B790000362036A23F400730362036A948843EA32
:10B7A00004230362294B984202D0294B984223D1AB
:10B7B000036A23F480630362036A548843EA042320
:10B7C0000362036A23F400630362036AD48843EAD2
:10B7D00004230362436823F480534360436814895D
:10B7E00043EA04134360436823F40053436043680F
:10B7F000548943EA0413436026E0036A23F4805328
:10B800000362C36923F44073C361036A148843EA83
:10B8100004330362036A23F400530362036A9488C7
:10B8200043EA04330362094B984202D0084B984222
:10B8300008D1436823F4804343604368148943EA92
:10B840008413436000E000BF00BF10BD002C014026
:10B850000034014031B101290CD0022913D0032951
:10B8600022D118E0836923F0700383618369134355
:10B8700083611AE0836923F4E0438361836943EAC7
:10B880000223836111E0C36923F07003C361C369BC
:10B890001343C36109E0C36923F4E043C361C3698F
:10B8A00043EA0223C36100E000BF00BF704731B12B
:10B8B000012906D0022906D0032908D105E04263F8
:10B8C00006E0826304E0C26302E0026400E000BFBD
:10B8D00000BF704731B101290CD0022913D00329D0
:10B8E00022D118E0836923F008038361836913433D
:10B8F00083611AE0836923F400638361836943EA07
:10B900000223836111E0C36923F00803C361C369A3
:10B910001343C36109E0C36923F40063C361C369CE
:10B9200043EA0223C36100E000BF00BF7047014645
:10B930000020486A704741627047000010B5044615
:10B940003349601A8C4244D00CDCB4F1804F1CD0D7
:10B950003048204410B3B0F5806F28D0B0F5006FA8
:10B9600052D12DE0B0F5806F3CD0B0F58E3F03D0C2
:10B97000B0F5923F48D13EE040F20B30FFF740FD7A
:10B9800040F20B30FFF72CFD3FE04FF48060FFF7F3
:10B9900037FD4FF48060FFF723FD36E040F20140B1
:10B9A000FFF72EFD40F20140FFF71AFD2DE040F2B7
:10B9B0000240FFF725FD40F20240FFF711FD24E0B1
:10B9C00040F20340FFF71CFD40F20340FFF708FD83
:10B9D0001BE040F20440FFF713FD40F20440FFF784
:10B9E000FFFC12E040F20540FFF70AFD40F205407F
:10B9F000FFF7F6FC09E040F20D30FFF701FD40F2E1
:10BA00000D30FFF7EDFC00E000BF00BF10BD0000EF
:10BA10000010004000FCFFBF016821F0010101603F
:10BA20007047016841F00101016070470A88826235
:10BA3000294A904220D0B0F1804F1DD0274A904231
:10BA40001AD0274A904217D0264A904214D0264A4C
:10BA5000904211D0254A90420ED0254A90420BD0F8
:10BA6000244A904208D0244A904205D0234A90426A
:10BA700002D0234A90420FD1026822F07002026085
:10BA800002688B7803F060031A43026002680B7946
:10BA900003F010031A4302608A68C262194A904296
:10BAA0000CD0194A904209D0026822F44072026018
:10BAB00002688B8903F440731A430260064A90427D
:10BAC00002D0094A904201D18A7B0263426942F066
:10BAD0000102426170470000002C01400004004058
:10BAE00000080040000C004000340140004C0140C0
:10BAF000005001400054014000180040001C00406C
:10BB0000002000400010004000140040C2688A433A
:10BB1000C2607047C2680A43C260704702698A43C4
:10BB2000026170470246D06800EA010310690840CC
:10BB300010B10BB1012070470020FCE7002101800B
:10BB4000418081804FF6FF71816000218181817386
:10BB5000704700002DE9F04704460D460027B8461F
:10BB6000B94600261D49601A8C421CD006DC1C48D0
:10BB7000204470B1B0F5806F1FD10FE0B0F5806F39
:10BB800016D0B0F56C4F18D10320FFF7F5FA074631
:10BB900014E00220FFF7F0FA07460FE00220FFF75B
:10BBA000EBFA07460AE00220FFF7E6FA074605E04F
:10BBB0000220FFF7E1FA074600E000BF00BF07EBF5
:10BBC0005500B0FBF5F64FF6F07006EA000806F0F7
:10BBD0000F0948EA0900A060BDE8F087004C00406A
:10BBE00000BCFFBF01464868C0F308007047C1F3BE
:10BBF000080242607047000010B504462049601AF0
:10BC00008C4228D006DC1F48204490B1B0F5806FEC
:10BC100033D117E0B0F5806F26D0B0F56C4F2CD142
:10BC200040F20E30FFF7ECFB40F20E30FFF7D8FB8E
:10BC300024E040F21140FFF7E3FB40F21140FFF730
:10BC4000CFFB1BE040F21240FFF7DAFB40F212405C
:10BC5000FFF7C6FB12E040F21340FFF7D1FB40F2C2
:10BC60001340FFF7BDFB09E040F21440FFF7C8FBAB
:10BC700040F21440FFF7B4FB00E000BF00BF10BD6E
:10BC8000004C004000BCFFBFC16841F40051C160DE
:10BC9000704710B5024602EB9110006801F01F04D6
:10BCA0000123A340184008B1012010BD0020FCE78B
:10BCB0000A460021416921F4007111434161704736
:10BCC0000A460021416921F48071114341617047A6
:10BCD00010B5C1F38912825801F01F040123A3405B
:10BCE0009A43C1F38913C25010BD10B5C1F3891234
:10BCF000825801F01F040123A3401A43C1F38913A2
:10BD0000C25010BD70B5024600230024C1F3891053
:10BD1000105801F01F060125B54000EA050302EBAB
:10BD200091500068C1F304460125B54000EA0504BE
:10BD300014B10BB1012070BD0020FCE7C26822F4F1
:10BD4000C062C260C2680A43C26070470A460021EE
:10BD5000C16821F004011143C1607047026922F4F7
:10BD60004052026102690A43026170470A4600219B
:10BD7000C16821F008011143C1607047C26822F414
:10BD80008052C260C2680A43C260704720F682F5E2
:10BD9000DCF42EF478F3B9F2F1F120F145F061EF23
:10BDA00073EE7AED77EC69EB51EA2DE9FEE7C4E634
:10BDB0007EE52CE4CFE266E1F0DF6FDEE2DC48DB1B
:10BDC000A3D9F1D734D66AD495D2B4D0C8CED1CCC9
:10BDD000CFCAC1C8AAC688C45DC228C0E9BDA3BB7A
:10BDE00054B9FDB69FB43AB2CFAF5EADE8AA6DA824
:10BDF000EEA56BA3E5A05D9ED39B4799BB962E94C1
:10BE0000A291178F8C8C048A7E87FB847C820080B1
:10BE1000887D167BA8783F76DD7381712B6FDC6C93
:10BE2000946A53681A66E863BF619E5F855D745BC0
:10BE30006C596D5776558953A451C84FF44D2A4C0F
:10BE4000694AB04801475A45BC4327429A40163FC9
:10BE50009A3D273CBC3A5939FE37AC3661351D3422
:10BE6000E232AD3180305B2F3C2E242D132C092B78
:10BE7000052A0829112820273526502571249723C3
:10BE8000C222F4212A216520A8BE0008000000205B
:10BE9000F800000064980008A0BF0008F800002027
:10BEA000C03100007498000800000000000000008D
:10BEB000000000000000010101000000000000007F
:10BEC0000000000000000100000031000000000040
:10BED0000000000031000000000000000000000031
:10BEE0000000000000000000000000000000000052
:10BEF00000000000FFFFFFFF000000000000000046
:10BF00000000000000000000000000000000000031
:10BF10000000000000000000000000000000000021
:10BF20000000000000000000000000000000000011
:10BF3000D2C6B75900000000140E0100FC0F01002A
:10BF400014160100000000000000000000000000C6
:10BF500000000000000000000000000000000000E1
:10BF600000000000000000000000000000000000D1
:10BF700000000000000000000000000000000000C1
:10BF800000000000000000000000000000000000B1
:10BF9000000000000000000000F36F060000000039
:00000001FF
